:020000040000FA
:0408000055EF0BF0B5
:1008100003B272EF05F0F2B490EF05F09EB098EFDE
:1008200005F09EB2A0EF05F0F2A81AEF04F0F2B2C4
:1008300021EF04F0F2B01FEF04F004EF0BF0F2969A
:10084000F290CD90F2929EA02BEF04F00101533F65
:100850002BEF04F0542BAEC1B2F1AFC1B3F1B0C174
:10086000B4F1B1C1B5F1AAC1AEF1ABC1AFF1ACC148
:10087000B0F1ADC1B1F1A6C1AAF1A7C1ABF1A8C158
:10088000ACF1A9C1ADF1A2C1A6F1A3C1A7F1A4C168
:10089000A8F1A5C1A9F19EC1A2F19FC1A3F1A0C178
:1008A000A4F1A1C1A5F19AC19EF19BC19FF19CC188
:1008B000A0F19DC1A1F196C19AF197C19BF198C198
:1008C0009CF199C19DF1CECF96F1CFCF97F153C155
:1008D00098F154C199F1CF6ACE6A0101536B546B00
:1008E0009E90CD800FBC0F8E0FBA7AEF04F00F8A66
:1008F00004EF0BF00F8C0FBEB6EF04F096C19AF127
:1009000097C19BF198C19CF199C19DF19AC19EF14B
:100910009BC19FF19CC1A0F19DC1A1F19EC1A2F11B
:100920009FC1A3F1A0C1A4F1A1C1A5F1A2C1A6F1EB
:10093000A3C1A7F1A4C1A8F1A5C1A9F1A6C1AAF1BB
:10094000A7C1ABF1A8C1ACF1A9C1ADF1AAC1AEF18B
:10095000ABC1AFF1ACC1B0F1ADC1B1F1AEC1B2F15B
:10096000AFC1B3F1B0C1B4F1B1C1B5F101015E6B7A
:100970005F6B606B616B96515E2797515F23985157
:100980006023995161239A515E279B515F239C51AB
:1009900060239D5161239E515E279F515F23A0518B
:1009A0006023A1516123A2515E27A3515F23A4516B
:1009B0006023A5516123A6515E27A7515F23A8514B
:1009C0006023A9516123AA515E27AB515F23AC512B
:1009D0006023AD516123AE515E27AF515F23B0510B
:1009E0006023B1516123B2515E27B3515F23B451EB
:1009F0006023B5516123D8900101613360335F33C7
:100A00005E33D8900101613360335F335E33D89039
:100A10000101613360335F335E3300C10CF101C10A
:100A20000DF102C10EF103C10FF104C110F105C1B6
:100A300011F106C112F107C113F108C114F109C186
:100A400015F10AC116F10BC117F134C135F111B816
:100A500035EF05F00101620E046F010E056F000E07
:100A6000066F000E076F3EEF05F00101A70E046F41
:100A7000020E056F000E066F000E076F5EC100F1DB
:100A80005FC101F160C102F161C103F138EC2CF0EA
:100A900003BF04D019BE02D019A0108C11A056EFCC
:100AA00005F010BA56EF05F00F80108A0CC100F166
:100AB0000DC101F10EC102F10FC103F110C104F12A
:100AC00011C105F112C106F113C107F114C108F1FA
:100AD00015C109F116C10AF117C10BF135C134F185
:100AE00004EF0BF00392ABB2AB98AB88030103EEBB
:100AF00000F080517F0BE92604C0EFFF802B81516D
:100B0000805D700BD8A48B8200008051815D700BDA
:100B1000D8A48B9281518019D8B4079004EF0BF0C0
:100B2000F2940101453F04EF0BF0462B04EF0BF06C
:100B30009E900101533F04EF0BF0542B04EF0BF098
:100B40009E9211B823EF08F0040066A1A8EF05F00B
:100B50008BB4B2EF05F010ACB2EF05F08B84109CB3
:100B6000B3EF05F08B94077C07ACCEEF05F0C274B1
:100B7000C2B4C8EF05F0C3CFB7F5C4CFB8F50501CF
:100B8000D890B833B733D890B833B733CFEF05F038
:100B9000C3CF55F1C4CF56F1CFEF05F0C28207B4F1
:100BA0003CEF06F047C14BF148C14CF149C14DF152
:100BB0004AC14EF15EC162F15FC163F160C164F18F
:100BC00061C165F196C1B6F197C1B7F198C1B8F1AD
:100BD00099C1B9F19AC1BAF19BC1BBF19CC1BCF1F9
:100BE0009DC1BDF19EC1BEF19FC1BFF1A0C1C0F1C9
:100BF000A1C1C1F1A2C1C2F1A3C1C3F1A4C1C4F199
:100C0000A5C1C5F1A6C1C6F1A7C1C7F1A8C1C8F168
:100C1000A9C1C9F1AAC1CAF1ABC1CBF1ACC1CCF138
:100C2000ADC1CDF1AEC1CEF1AFC1CFF1B0C1D0F108
:100C3000B1C1D1F1B2C1D2F1B3C1D3F1B4C1D4F1D8
:100C4000B5C1D5F1B7C5B9F5B8C5BAF5B9C5BBF5E4
:100C5000BAC5BCF5010155515B2756515C23E86AC2
:100C60005D230E2E3CEF06F05CC157F15DC158F1DB
:100C70005B6B5C6B5D6B078E0201002F04EF0BF06A
:100C80003C0E006F1A50E00BE00AE866128818BEAE
:100C900002D018B4108E00C10CF101C10DF102C1D7
:100CA0000EF103C10FF104C110F105C111F106C12C
:100CB00012F107C113F108C114F109C115F10AC1FC
:100CC00016F10BC117F134C135F181AA1CEF07F001
:100CD00030A0EDEF06F005012F51000AD8B41CEF4B
:100CE00007F005012F51010AD8B4A6EF06F005015F
:100CF0002F51020AD8B4E7EF06F005012F51030A7D
:100D0000D8B4E7EF06F005012F51040AD8B4E7EF95
:100D100006F005012F51050AD8B4E7EF06F00501EA
:100D20002F51060AD8B4E7EF06F005012F51070A44
:100D3000D8B4E7EF06F005012F51320AD8B4A4EF7A
:100D400006F02F6B1CEF07F01CEF07F0050157674B
:100D5000B1EF06F05867B1EF06F05967B1EF06F052
:100D60005A67B5EF06F01CEF07F05BC500F15CC5F4
:100D700001F15DC502F15EC503F10101010E046FD1
:100D8000000E056F000E066F000E076F38EC2CF09A
:100D900000C15BF501C15CF502C15DF503C15EF503
:100DA0000067DAEF06F00167DAEF06F00267DAEFC4
:100DB00006F003671CEF07F057C55BF558C55CF5F7
:100DC00059C55DF55AC55EF50F881CEF07F00501A2
:100DD0003067EDEF06F01CEF07F00FBE02EF07F0F3
:100DE00010A007EF07F001014767FEEF06F0486724
:100DF000FEEF06F04967FEEF06F04A6702EF07F0E4
:100E000007EF07F007AE07EF07F019EF07F005014E
:100E1000312F1CEF07F03C0E316F302F1CEF07F025
:100E20000101000E626FE00E636FA50E646F010E8C
:100E3000656F0501306B0F880501666B37B722EFD0
:100E400007F066810CC100F10DC101F10EC102F184
:100E50000FC103F110C104F111C105F112C106F176
:100E600013C107F114C108F115C109F116C10AF146
:100E700017C10BF135C134F100C10CF101C10DF105
:100E800002C10EF103C10FF104C110F105C111F14E
:100E900006C112F107C113F108C114F109C115F11E
:100EA0000AC116F10BC117F134C135F101018A678E
:100EB00061EF07F08B6761EF07F08C6761EF07F078
:100EC0008D6765EF07F095EF07F08EC100F18FC1D8
:100ED00001F190C102F191C103F10101010E046F12
:100EE000000E056F000E066F000E076F38EC2CF039
:100EF00000C18EF101C18FF102C190F103C191F1E6
:100F000000678AEF07F001678AEF07F002678AEF50
:100F100007F0036795EF07F08AC18EF18BC18FF15F
:100F20008CC190F18DC191F10F80D57ED5BE6DD071
:100F3000D6CF47F1D7CF48F145C149F1E86AE8CFAC
:100F40004AF119BE02D019A0108C109047C100F1CF
:100F500048C101F149C102F14AC103F101010A0E80
:100F6000046F000E056F000E066F000E076F38EC61
:100F70002CF003AF1080010154A7CBEF07F00F9ABC
:100F80000F9C0F9E0101000E5E6F600E5F6F3D0EA5
:100F9000606F080E616F010147BFDBEF07F0486724
:100FA000DBEF07F04967DBEF07F04A67DBEF07F09D
:100FB000F28800EF08F0F2985E6B5F6B606B616B1C
:100FC000966B976B986B996B9A6B9B6B9C6B9D6BFD
:100FD0009E6B9F6BA06BA16BA26BA36BA46BA56BAD
:100FE000A66BA76BA86BA96BAA6BAB6BAC6BAD6B5D
:100FF000AE6BAF6BB06BB16BB26BB36BB46BB56B0D
:10100000D76AD66A0101456B466B0CC100F10DC170
:1010100001F10EC102F10FC103F110C104F111C1C0
:1010200005F112C106F113C107F114C108F115C190
:1010300009F116C10AF117C10BF135C134F104EF02
:101040000BF004EF0BF00201002F6DEF0AF0D59EBC
:10105000D6CF47F1D7CF48F145C149F1E86AE8CF8B
:101060004AF1D76AD66A0101456B466BD58E1A5094
:10107000E00BE00AE866128818BE02D018B4108EA1
:1010800017AE1C8C00C10CF101C10DF102C10EF1B3
:1010900003C10FF104C110F105C111F106C112F134
:1010A00007C113F108C114F109C115F10AC116F104
:1010B0000BC117F134C135F10FA0109A11B86CEFC4
:1010C00008F00101620E046F010E056F000E066F3D
:1010D000000E076F75EF08F00101A70E046F020EF6
:1010E000056F000E066F000E076F47C100F148C183
:1010F00001F149C102F14AC103F138EC2CF003BF00
:1011000088EF08F019BE02D019A0108C11B00F8022
:101110000CC100F10DC101F10EC102F10FC103F1CB
:1011200010C104F111C105F112C106F113C107F19B
:1011300014C108F115C109F116C10AF117C10BF16B
:1011400035C134F102013C0E006F00C10CF101C148
:101150000DF102C10EF103C10FF104C110F105C17F
:1011600011F106C112F107C113F108C114F109C14F
:1011700015F10AC116F10BC117F134C135F181AA7D
:1011800076EF09F030A047EF09F005012F51000A72
:10119000D8B476EF09F005012F51010AD8B400EF59
:1011A00009F005012F51020AD8B441EF09F00501F9
:1011B0002F51030AD8B441EF09F005012F51040A59
:1011C000D8B441EF09F005012F51050AD8B441EF19
:1011D00009F005012F51060AD8B441EF09F00501C5
:1011E0002F51070AD8B441EF09F005012F51320AF7
:1011F000D8B4FEEF08F02F6B76EF09F076EF09F028
:10120000050157670BEF09F058670BEF09F05967B5
:101210000BEF09F05A670FEF09F076EF09F05BC5A5
:1012200000F15CC501F15DC502F15EC503F101018C
:10123000010E046F000E056F000E066F000E076FA3
:1012400038EC2CF000C15BF501C15CF502C15DF525
:1012500003C15EF5006734EF09F0016734EF09F070
:10126000026734EF09F0036776EF09F057C55BF5C5
:1012700058C55CF559C55DF55AC55EF50F8876EF22
:1012800009F00501306747EF09F076EF09F00FBE6E
:101290005CEF09F010A061EF09F00101476758EF1A
:1012A00009F0486758EF09F0496758EF09F04A67B5
:1012B0005CEF09F061EF09F007AE61EF09F073EF41
:1012C00009F00501312F76EF09F03C0E316F302F18
:1012D00076EF09F00101000E626FE00E636FA50E5C
:1012E000646F010E656F0501306B0F880501666B39
:1012F00037B77CEF09F066810CC100F10DC101F137
:101300000EC102F10FC103F110C104F111C105F1C9
:1013100012C106F113C107F114C108F115C109F199
:1013200016C10AF117C10BF135C134F100C10CF13E
:1013300001C10DF102C10EF103C10FF104C110F1A1
:1013400005C111F106C112F107C113F108C114F171
:1013500009C115F10AC116F10BC117F134C135F1FC
:1013600001018A67BBEF09F08B67BBEF09F08C675F
:10137000BBEF09F08D67BFEF09F0EFEF09F08EC109
:1013800000F18FC101F190C102F191C103F101019E
:10139000010E046F000E056F000E066F000E076F42
:1013A00038EC2CF000C18EF101C18FF102C190F137
:1013B00003C191F10067E4EF09F00167E4EF09F080
:1013C0000267E4EF09F00367EFEF09F08AC18EF1DD
:1013D0008BC18FF18CC190F18DC191F10F80109074
:1013E00047C100F148C101F149C102F14AC103F10D
:1013F00001010A0E046F000E056F000E066F000E4D
:10140000076F38EC2CF003AF1080010154A715EFE3
:101410000AF00F9A0F9C0F9E0101000E5E6F600E86
:101420005F6F3D0E606F080E616F47C100F148C1EC
:1014300001F149C102F14AC103F10101140E046F27
:10144000050E056F000E066F000E076F38EC2CF0CE
:1014500003AF2EEF0AF0F28853EF0AF0F2985E6BBA
:101460005F6B606B616B966B976B986B996B9A6B0C
:101470009B6B9C6B9D6B9E6B9F6BA06BA16BA26B20
:10148000A36BA46BA56BA66BA76BA86BA96BAA6BD0
:10149000AB6BAC6BAD6BAE6BAF6BB06BB16BB26B80
:1014A000B36BB46BB56B0CC100F10DC101F10EC192
:1014B00002F10FC103F110C104F111C105F112C114
:1014C00006F113C107F114C108F115C109F116C1E4
:1014D0000AF117C10BF135C134F104008BB478EF78
:1014E0000AF010AC78EF0AF08B84109C79EF0AF0C8
:1014F0008B94077C07AC94EF0AF0C274C2B48EEFF1
:101500000AF0C3CFB7F5C4CFB8F50501D890B8330A
:10151000B733D890B833B73395EF0AF0C3CF55F14E
:10152000C4CF56F195EF0AF0C28207B402EF0BF078
:1015300047C14BF148C14CF149C14DF14AC14EF18F
:101540005EC162F15FC163F160C164F161C165F1C7
:1015500096C1B6F197C1B7F198C1B8F199C1B9F187
:101560009AC1BAF19BC1BBF19CC1BCF19DC1BDF157
:101570009EC1BEF19FC1BFF1A0C1C0F1A1C1C1F127
:10158000A2C1C2F1A3C1C3F1A4C1C4F1A5C1C5F1F7
:10159000A6C1C6F1A7C1C7F1A8C1C8F1A9C1C9F1C7
:1015A000AAC1CAF1ABC1CBF1ACC1CCF1ADC1CDF197
:1015B000AEC1CEF1AFC1CFF1B0C1D0F1B1C1D1F167
:1015C000B2C1D2F1B3C1D3F1B4C1D4F1B5C1D5F137
:1015D000B7C5B9F5B8C5BAF5B9C5BBF5BAC5BCF557
:1015E000010155515B2756515C23E86A5D230E2E9D
:1015F00002EF0BF05CC157F15DC158F15B6B5C6BA6
:101600005D6B078E04EF0BF002C0E0FF005001C0DD
:10161000D8FF1000A6B20AEF0BF00CC0A9FF0BC058
:10162000A8FFA69EA69CA684F29E550EA76EAA0EA3
:10163000A76EA682F28EA694A6B21CEF0BF00C2A1F
:101640001200A96EA69EA69CA680A8500C2A120085
:1016500004012C0E826F73EC0EF033EC2DF00C5065
:1016600021EC0BF0E8CF00F10C5021EC0BF0E8CFAF
:1016700001F101AF41EF0BF00101FF0E026FFF0E10
:10168000036FD6EC2CF029674DEF0BF00401200E10
:10169000826F73EC0EF052EF0BF004012D0E826F8F
:1016A00073EC0EF0E0EC2AF01200306A076A0F6A61
:1016B000106A116A126A136A0F010D0EC16E860E4E
:1016C000C06E030EC26E0F01680E896E130E926E0D
:1016D000080E8A6EF30E936E8B6A900E946EC80E8F
:1016E00021EC0BF0E8CFE8FF1098E8A0108810A8D4
:1016F00005D00E0E226E8E0E236E04D00F0E226EBB
:101700008F0E236EB2EC2DF0F18EF19EFC0E21ECCB
:101710000BF0E8CF0BF00BA011800BA211820BA4F1
:1017200011840BA81188C90E21EC0BF0E8CF17F03B
:10173000CA0E21EC0BF0E8CF18F0CB0E21EC0BF029
:10174000E8CF19F0CC0E21EC0BF0E8CF1AF0CD0E5B
:1017500021EC0BF0E8CF2FF01C6A1D6A0E6A010124
:101760005B6B5C6B5D6B576B586BF29A0101476B5F
:10177000486B496B4A6B4B6B4C6B4D6B4E6B4F6BB5
:10178000506B516B526B456B466BD76AD66A0F0133
:10179000280ED56EF28A9D90B00ECD6E01015E6B63
:1017A0005F6B606B616B626B636B646B656B666BCD
:1017B000676B686B696B536B546BCF6ACE6A0F9A19
:1017C0000F9C0F9E9D80760ECA6E9D8202013C0E7C
:1017D000006FCC6A160E21EC0BF0E8CF00F1170E6B
:1017E00021EC0BF0E8CF01F1180E21EC0BF0E8CF63
:1017F00002F1190E21EC0BF0E8CF03F1010103AF68
:101800001CEF0CF033EC2DF0160E0C6E00C10BF03B
:101810000AEC0BF0170E0C6E01C10BF00AEC0BF08A
:10182000180E0C6E02C10BF00AEC0BF0190E0C6EC8
:1018300003C10BF00AEC0BF000C18AF101C18BF17E
:1018400002C18CF103C18DF100C18EF101C18FF194
:1018500002C190F103C191F11A0E21EC0BF0E8CF17
:1018600000F11B0E21EC0BF0E8CF01F11C0E21EC76
:101870000BF0E8CF02F11D0E21EC0BF0E8CF03F1E5
:10188000010103AF72EF0CF033EC2DF01A0E0C6E69
:1018900000C10BF00AEC0BF01B0E0C6E01C10BF03B
:1018A0000AEC0BF01C0E0C6E02C10BF00AEC0BF0F4
:1018B0001D0E0C6E03C10BF00AEC0BF01A0E21EC9E
:1018C0000BF0E8CF00F11B0E21EC0BF0E8CF01F19B
:1018D0001C0E21EC0BF0E8CF02F11D0E21EC0BF0F9
:1018E000E8CF03F100C192F101C193F102C194F17B
:1018F00003C195F1240EAC6E900EAB6E240EAC6E4F
:10190000080EB86E000EB06E1F0EAF6E0401806B35
:10191000816B0F01900EAB6E0F019D8A0301806BEE
:10192000816BC26B8B9256EC32F056EC32F0B4EC19
:1019300033F035EC30F0200E21EC0BF0E8CF2FF532
:1019400005012F51FF0AD8A4ADEF0CF02F6B200E2C
:101950000C6E2FC50BF00AEC0BF00501010E306F79
:101960003C0E316F250E21EC0BF0E8CF00F1260E76
:1019700021EC0BF0E8CF01F1270E21EC0BF0E8CFC2
:1019800002F1280E21EC0BF0E8CF03F1010103AFC7
:10199000E4EF0CF033EC2DF0250E0C6E00C10BF0D3
:1019A0000AEC0BF0260E0C6E01C10BF00AEC0BF0EA
:1019B000270E0C6E02C10BF00AEC0BF0280E0C6E19
:1019C00003C10BF00AEC0BF000C157F501C158F54B
:1019D00002C159F503C15AF500C15BF501C15CF5BF
:1019E00002C15DF503C15EF5290E21EC0BF0E8CFD5
:1019F0005FF5050160515F5DD8A05FC560F5210E00
:101A000021EC0BF0E8CF00F1220E21EC0BF0E8CF37
:101A100001F1230E21EC0BF0E8CF02F1240E21ECB2
:101A20000BF0E8CF03F1010103AF45EF0DF033EC0C
:101A30002DF0210E0C6E00C10BF00AEC0BF0220E03
:101A40000C6E01C10BF00AEC0BF0230E0C6E02C100
:101A50000BF00AEC0BF0240E0C6E03C10BF00AEC39
:101A60000BF0210E21EC0BF0E8CF00F1220E21EC5F
:101A70000BF0E8CF01F1230E21EC0BF0E8CF02F1DF
:101A8000240E21EC0BF0E8CF03F100C161F501C198
:101A900062F502C163F503C164F57DEC2FF063ECE0
:101AA0002EF0BBEC2DF030A0B6EF0DF005012F515C
:101AB000020A16E005012F51030A19E005012F5112
:101AC000040A24E005012F51050A2BE005012F51DE
:101AD000060A39E005012F51070A3FE0B6EF0DF085
:101AE000602FB3EF0DF05FC560F5B6EF0DF0B0C538
:101AF00000F101010F0E001701010051000A36E04C
:101B000001010051050A32E0B3EF0DF0B0C500F15C
:101B100001010F0E001701010051000A27E0B3EF89
:101B20000DF00501B051000A21E00501B051150A80
:101B30001DE00501B051300A19E00501B051450A18
:101B400015E0B3EF0DF00501B051000A0FE00501FB
:101B5000B051300A0BE0B3EF0DF00501B051000AAF
:101B600005E0B3EF0DF081BAF3EF33F00790000119
:101B7000F28EF28C12AE03D012BCB2EF18F007B0A6
:101B800066EF29F00FB0FEEF22F010BEFEEF22F05C
:101B900012B8FEEF22F00FB89AEF1CF0030180514B
:101BA00081197F0BD8B466EF29F013EE00F0815154
:101BB0007F0BE126812BE7CFE8FFE00BD8B466EF7F
:101BC00029F023EE82F0C2513F0BD926E7CFDFFF89
:101BD000C22BDF50780AD8A466EF29F007808EC1A7
:101BE00000F18FC101F190C102F191C103F1010136
:101BF000040E046F000E056F000E066F000E076FD7
:101C000038EC2CF000AF0EEF0EF00101030E8E6FDA
:101C1000000E8F6F000E906F000E916F03018251C6
:101C2000720AD8B4E3EF22F08251520AD8B4E3EF3B
:101C300022F08251750AD8B4E3EF22F08251630A90
:101C4000D8B420EF26F08251690AD8B492EF1FF081
:101C500082517A0AD8B4A5EF20F08251490AD8B44B
:101C600031EF1FF08251500AD8B44FEF1EF082516D
:101C7000700AD8B492EF1EF08251540AD8B4BDEF66
:101C80001EF08251740AD8B403EF1FF08251410A4A
:101C9000D8B489EF0FF082514B0AD8B487EF0EF019
:101CA00082516D0AD8B4BCEF13F082514D0AD8B4FA
:101CB000D5EF13F08251730AD8B413EF22F082519A
:101CC000530AD8B478EF22F082514C0AD8B464EFAA
:101CD00014F08251590AD8B40DEF13F012AE01D0AE
:101CE000128C57EF26F0040114EE00F080517F0BA8
:101CF000E12682C4E7FF802B120004010D0E826FE3
:101D000073EC0EF00A0E826F73EC0EF012000401F9
:101D10004B0E826F73EC0EF004012C0E826F73EC8D
:101D20000EF081B802D02FB630D003018351430AA0
:101D3000D8B4CCEF0EF003018351630AD8B4CEEFD0
:101D40000EF003018351520AD8B4D0EF0EF0030114
:101D50008351720AD8B4D2EF0EF003018351470ABF
:101D6000D8B4D4EF0EF003018351670AD8B4D6EF8C
:101D70000EF003018351540AD8B4D8EF0EF00301DA
:101D80008351740AD8B447EF0FF003018351550A09
:101D9000D8B4DAEF0EF082D02F807AD02F9078D09E
:101DA0002F8276D02F9274D02F8472D02F9470D03F
:101DB0002F866ED084C330F185C331F186C332F1F2
:101DC00087C333F10101296B81EC2DF0F8EC2CF085
:101DD00000C104F101C105F102C106F103C107F11F
:101DE00074EC2DF0200EF86EF76AF66A0900F5CF54
:101DF0002CF10900F5CF2DF10900F5CF2EF10900E6
:101E0000F5CF2FF10900F5CF30F10900F5CF31F111
:101E10000900F5CF32F10900F5CF33F10101296B4B
:101E200081EC2DF0F8EC2CF038EC2CF0006720EF72
:101E30000FF0016720EF0FF0026720EF0FF003674C
:101E400001D025D004014E0E826F73EC0EF0040118
:101E50006F0E826F73EC0EF004014D0E826F73EC07
:101E60000EF00401610E826F73EC0EF00401740E2B
:101E7000826F73EC0EF00401630E826F73EC0EF050
:101E80000401680E826F73EC0EF055EF26F02F966A
:101E9000CD0E0C6E2FC00BF00AEC0BF0CD0E21EC2A
:101EA0000BF0E8CF2FF02FB006D00401630E826F45
:101EB00073EC0EF005D00401430E826F73EC0EF04C
:101EC0002FB206D00401720E826F73EC0EF005D0B3
:101ED0000401520E826F73EC0EF02FB406D0040191
:101EE000670E826F73EC0EF005D00401470E826F0F
:101EF00073EC0EF02FB606D00401740E826F73ECF3
:101F00000EF005D00401540E826F73EC0EF055EF05
:101F100026F00401410E826F73EC0EF00301835131
:101F2000310AD8B42DEF12F003018351320AD8B42C
:101F30005DEF11F003018351330AD8B4E6EF10F0DE
:101F400003018351340AD8B4D6EF0FF00301835153
:101F5000350AD8B4B3EF0FF004013F0E826F73EC73
:101F60000EF055EF26F004012C0E826F73EC0EF08C
:101F700003018451300AD8B4C6EF0FF00301845135
:101F8000310AD8B4CEEF0FF01FEF11F08B9004019F
:101F9000300E826F73EC0EF0D4EF0FF08B800401E3
:101FA000310E826F73EC0EF055EF26F0CC0E21EC63
:101FB0000BF0E8CF0BF004012C0E826F73EC0EF0E7
:101FC00003018451310AD8B4FAEF0FF003018451B0
:101FD000300AD8B4FCEF0FF0030184514D0AD8B495
:101FE00006EF10F003018451540AD8B40DEF10F03D
:101FF00024EF10F08A8401D08A940BAE04D00BAC8D
:1020000002D00BBA21D0E00E0B1218D01F0E0B1607
:102010008539E844E00B0B1211D0E00E0B1674EC7E
:102020002DF085C332F186C333F10101296B81ECB8
:102030002DF0F8EC2CF000511F0B0B12CC0E0C6E97
:102040000BC00BF00AEC0BF00401340E826F73EC42
:102050000EF004012C0E826F73EC0EF0CC0E21EC0E
:102060000BF0E8CF1AF08AB406D00401300E826F6C
:1020700073EC0EF005D00401310E826F73EC0EF09C
:1020800004012C0E826F73EC0EF01A38E840070B37
:10209000E8CF82F40401300E822773EC0EF00401C5
:1020A0002C0E826F73EC0EF033EC2DF01A501F0BD8
:1020B000E8CF00F1D6EC2CF032C182F40401300EEE
:1020C000822773EC0EF033C182F40401300E8227B4
:1020D00073EC0EF004012C0E826F73EC0EF033ECF7
:1020E0002DF02DC000F100AF0BD0FF0E016FFF0EE1
:1020F000026FFF0E036F04012D0E826F73EC0EF062
:10210000D6EC2CF031C182F40401300E822773EC3E
:102110000EF032C182F40401300E822773EC0EF00F
:1021200033C182F40401300E822773EC0EF00401F7
:102130002C0E826F73EC0EF033EC2DF02CC000F1FE
:10214000D6EC2CF031C182F40401300E822773ECFE
:102150000EF032C182F40401300E822773EC0EF0CF
:1021600033C182F40401300E822773EC0EF00401B7
:102170002C0E826F73EC0EF033EC2DF02EC000F1BC
:1021800000AF0BD0FF0E016FFF0E026FFF0E036F4B
:1021900004012D0E826F73EC0EF0D6EC2CF031C1E1
:1021A00082F40401300E822773EC0EF032C182F407
:1021B0000401300E822773EC0EF033C182F4040167
:1021C000300E822773EC0EF055EF26F0CB0E21EC8B
:1021D0000BF0E8CF0BF004012C0E826F73EC0EF0C5
:1021E00003018451450AD8B40AEF11F00301845168
:1021F000440AD8B40DEF11F003018451300AD8B469
:1022000010EF11F003018451310AD8B414EF11F02A
:102210001FEF11F00B9E19EF11F00B8E19EF11F05B
:10222000FC0E0B1619EF11F0FC0E0B160B8019EFBC
:1022300011F0CB0E0C6E0BC00BF00AEC0BF004018E
:10224000330E826F73EC0EF004012C0E826F73EC70
:102250000EF0CB0E21EC0BF0E8CF19F019BE38EFE1
:1022600011F00401450E826F73EC0EF03DEF11F09A
:102270000401440E826F73EC0EF004012C0E826F89
:1022800073EC0EF00401300E826F73EC0EF004015B
:102290002C0E826F73EC0EF019B056EF11F00401A2
:1022A000300E826F73EC0EF05BEF11F00401310E13
:1022B000826F73EC0EF055EF26F0CA0E21EC0BF096
:1022C000E8CF0BF004012C0E826F73EC0EF00301CB
:1022D0008451450AD8B499EF11F003018451440A9E
:1022E000D8B49CEF11F0030184514D0AD8B4A5EF86
:1022F00011F003018451410AD8B49FEF11F003019A
:102300008451460AD8B4A2EF11F003018451560A51
:10231000D8B4ADEF11F003018451500AD8B4B8EF2E
:1023200011F003018451520AD8B4BBEF11F0C4EF8D
:1023300011F00B9EBEEF11F00B8EBEEF11F00B9C57
:10234000BEEF11F00B8CBEEF11F0FC0E0B1685C327
:10235000E8FF030B0B12BEEF11F0C70E0B1685C37F
:10236000E8FF070BE846E846E8460B12BEEF11F01F
:102370000B84BEEF11F00B94BEEF11F0CA0E0C6E81
:102380000BC00BF00AEC0BF0CA0E21EC0BF0E8CFFF
:1023900018F00401320E826F73EC0EF004012C0E63
:1023A000826F73EC0EF018BEDDEF11F00401450EE4
:1023B000826F73EC0EF0E2EF11F00401440E826FB5
:1023C00073EC0EF004012C0E826F73EC0EF018C04B
:1023D000E8FF030BE8CF82F40401300E822773EC90
:1023E0000EF004012C0E826F73EC0EF018BC00EF9F
:1023F00012F00401410E826F73EC0EF005EF12F043
:102400000401460E826F73EC0EF004012C0E826FF5
:1024100073EC0EF018C0E8FF380BE842E842E842DF
:10242000E8CF82F40401300E822773EC0EF0040131
:102430002C0E826F73EC0EF018B426EF12F004012C
:10244000520E826F73EC0EF02BEF12F00401500E5F
:10245000826F73EC0EF055EF26F0C90E21EC0BF0F5
:10246000E8CF0BF004012C0E826F73EC0EF0030129
:102470008451450AD8B44BEF12F003018451440A49
:10248000D8B44EEF12F0030184514D0AD8B451EF85
:1024900012F05FEF12F00B9E59EF12F00B8E59EF16
:1024A00012F0F80E0B1685C3E8FF070B0B1259EF5D
:1024B00012F0C90E0C6E0BC00BF00AEC0BF004010D
:1024C000310E826F73EC0EF004012C0E826F73ECF0
:1024D0000EF0C90E21EC0BF0E8CF17F017BE06D0B6
:1024E0000401450E826F73EC0EF005D00401440E1A
:1024F000826F73EC0EF004012C0E826F73EC0EF001
:1025000017C0E8FF070BE8CF82F40401300E8227E2
:1025100073EC0EF004012C0E826F73EC0EF007804A
:1025200033EC2DF028C0E8FF003B00430043030BD1
:10253000D6EC2CF033C182F40401300E822773EC08
:102540000EF004012C0E826F73EC0EF033EC2DF0C4
:1025500028C001F1019F019D29C000F10101D6ECC5
:102560002CF02FC182F40401300E822773EC0EF0A0
:1025700030C182F40401300E822773EC0EF031C1B9
:1025800082F40401300E822773EC0EF032C182F423
:102590000401300E822773EC0EF033C182F4040183
:1025A000300E822773EC0EF004012C0E826F73EC58
:1025B0000EF033EC2DF02AC001F12BC000F1D890C1
:1025C00001330033D890013300330101D6EC2CF0F5
:1025D0002FC182F40401300E822773EC0EF030C15B
:1025E00082F40401300E822773EC0EF031C182F4C4
:1025F0000401300E822773EC0EF032C182F4040124
:10260000300E822773EC0EF033C182F40401300ED9
:10261000822773EC0EF055EF26F0FC0E21EC0BF048
:10262000E8CF0BF003018351520AD8B444EF13F002
:1026300003018351720AD8B447EF13F003018351A9
:10264000500AD8B44AEF13F003018351700AD8B48A
:102650004DEF13F003018351550AD8B450EF13F036
:1026600003018351750AD8B453EF13F0030183516A
:10267000430AD8B45CEF13F003018351630AD8B462
:102680005FEF13F068EF13F00B9062EF13F00B8025
:1026900062EF13F00B9262EF13F00B8262EF13F014
:1026A0000B9462EF13F00B8462EF13F00B9662EF62
:1026B00013F00B8662EF13F00B9862EF13F00B88A8
:1026C00062EF13F0FC0E0C6E0BC00BF00AEC0BF07B
:1026D0000401590E826F73EC0EF011901192119457
:1026E0001198FC0E21EC0BF0E8CF0BF00BA0118041
:1026F0000BA211820BA411840BA8118811A088EFE2
:1027000013F00401520E826F73EC0EF08DEF13F094
:102710000401720E826F73EC0EF011A897EF13F0A4
:102720000401430E826F73EC0EF09CEF13F0040172
:10273000630E826F73EC0EF011A2A6EF13F004018A
:10274000500E826F73EC0EF0ABEF13F00401700EBD
:10275000826F73EC0EF011A4B5EF13F00401550E67
:10276000826F73EC0EF0BAEF13F00401750E826FF6
:1027700073EC0EF055EF26F004016D0E826F73ECD2
:102780000EF003018351300AD8B414EF14F00301A2
:102790008351310AD8B427EF14F003018351320A70
:1027A000D8B43AEF14F057EF26F004014D0E826FC3
:1027B00073EC0EF074EC2DF084C331F185C332F16B
:1027C00086C333F10101296B81EC2DF0F8EC2CF07C
:1027D00003018351300AD8B4FCEF13F00301835195
:1027E000310AD8B404EF14F003018351320AD8B48B
:1027F0000CEF14F057EF26F0FD0E0C6E00C10BF03D
:102800000AEC0BF014EF14F0FE0E0C6E00C10BF08E
:102810000AEC0BF027EF14F0FF0E0C6E00C10BF06A
:102820000AEC0BF03AEF14F00401300E826F73ECF7
:102830000EF004012C0E826F73EC0EF033EC2DF0D1
:10284000FD0E21EC0BF0E8CF00F14BEF14F004018A
:10285000310E826F73EC0EF004012C0E826F73EC5C
:102860000EF033EC2DF0FE0E21EC0BF0E8CF00F172
:102870004BEF14F00401320E826F73EC0EF033EC68
:102880002DF004012C0E826F73EC0EF0FF0E21EC84
:102890000BF0E8CF00F1D6EC2CF031C182F404014A
:1028A000300E822773EC0EF032C182F40401300E38
:1028B000822773EC0EF033C182F40401300E8227BC
:1028C00073EC0EF055EF26F003018351300AD8B4B3
:1028D0005FEF19F003018351310AD8B48CEF1AF07D
:1028E00003018351320AD8B4FAEF1AF0030183517D
:1028F000330AD8B40AEF1BF003018351340AD8B469
:102900001AEF1BF003018351350AD8B4A0EF1CF075
:1029100003018351360AD8B4CEEF1CF00301835172
:10292000370AD8B437EF17F003018351380AD8B407
:10293000D5EF17F003018351460AD8B4F3EF1BF02B
:10294000030183514D0AD8B4B0EF15F00301835150
:102950006D0AD8B4CAEF15F0030183515A0AD8B4EE
:1029600006EF1AF003018351490AD8B4CEEF1DF0E7
:1029700003018351500AD8B400EF1DF003018351C5
:10298000540AD8B479EF1DF003018351630AD8B417
:10299000EAEF15F003018351430AD8B4E2EF16F0D1
:1029A00003018351730AD8B4E8EF15F00301835192
:1029B000610AD8B4FDEF14F003018351650AD8B45D
:1029C000AFEF19F003018351450AD8B4BDEF19F0F8
:1029D00003018351620AD8B4CBEF19F0030183518C
:1029E000420AD8B4D9EF19F003018351760AD8B45A
:1029F000E7EF19F0D8A457EF26F004014C0E826FD0
:102A000073EC0EF00401610E826F73EC0EF063EC58
:102A10002EF004012C0E826F73EC0EF033EC2DF0CF
:102A2000AFC500F10101D6EC2CF031C182F40401F4
:102A3000300E822773EC0EF032C182F40401300EA6
:102A4000822773EC0EF033C182F40401300E82272A
:102A500073EC0EF004012C0E826F73EC0EF033EC6D
:102A60002DF0B0C500F10101D6EC2CF031C182F49B
:102A70000401300E822773EC0EF032C182F404019F
:102A8000300E822773EC0EF033C182F40401300E55
:102A9000822773EC0EF004012C0E826F73EC0EF0A3
:102AA00033EC2DF0B1C500F10101D6EC2CF031C1B1
:102AB00082F40401300E822773EC0EF032C182F4EE
:102AC0000401300E822773EC0EF033C182F404014E
:102AD000300E822773EC0EF004012C0E826F73EC23
:102AE0000EF033EC2DF0B2C500F10101D6EC2CF064
:102AF00031C182F40401300E822773EC0EF032C132
:102B000082F40401300E822773EC0EF033C182F49C
:102B10000401300E822773EC0EF004012C0E826F3C
:102B200073EC0EF033EC2DF0B6C500F10101D6ECDC
:102B30002CF031C182F40401300E822773EC0EF0C8
:102B400032C182F40401300E822773EC0EF033C1DF
:102B500082F40401300E822773EC0EF0FCEF1CF0BF
:102B600074EC2DF084C333F181EC2DF0F8EC2CF0F3
:102B7000200E0C6E00C10BF00AEC0BF000C12FF51B
:102B800005012F51000A06E005012F51010A02E05C
:102B9000FDEC2EF004014C0E826F73EC0EF004017C
:102BA0004D0E826F73EC0EF004012C0E826F73ECED
:102BB0000EF033EC2DF02FC500F1D6EC2CF033C124
:102BC00082F40401300E822773EC0EF0FCEF1CF04F
:102BD000F3EF33F004014C0E826F73EC0EF004013E
:102BE000630E826F73EC0EF0BBEC2DF004012C0E23
:102BF000826F73EC0EF0FFEC15F0FCEF1CF033EC81
:102C00002DF0B5C500F10101003B0F0E0017D6EC09
:102C10002CF033C182F40401300E822773EC0EF0E5
:102C2000B5C500F101010F0E01010017D6EC2CF023
:102C300033C182F40401300E822773EC0EF00401DC
:102C40002D0E826F73EC0EF0B4C500F10101003B54
:102C50000F0E0017D6EC2CF033C182F40401300EB5
:102C6000822773EC0EF0B4C500F101010F0E0101D3
:102C70000017D6EC2CF033C182F40401300E822709
:102C800073EC0EF004012D0E826F73EC0EF0B3C5E1
:102C900000F10101003B0F0E0017D6EC2CF033C100
:102CA00082F40401300E822773EC0EF0B3C500F1FC
:102CB00001010F0E01010017D6EC2CF033C182F494
:102CC0000401300E822773EC0EF00401200E826F97
:102CD00073EC0EF0B2C500F10F0E01010017D6EC37
:102CE0002CF033C182F40401300E822773EC0EF015
:102CF0000401200E826F73EC0EF0B1C500F10101EA
:102D00000101003B0F0E0017D6EC2CF033C182F40A
:102D10000401300E822773EC0EF0B1C500F1010101
:102D20000F0E01010017D6EC2CF033C182F4040120
:102D3000300E822773EC0EF004013A0E826F73ECB2
:102D40000EF0B0C500F10101003B0F0E0017D6ECEC
:102D50002CF033C182F40401300E822773EC0EF0A4
:102D6000B0C500F101010F0E01010017D6EC2CF0E7
:102D700033C182F40401300E822773EC0EF004019B
:102D80003A0E826F73EC0EF0AFC500F10101003B0B
:102D90000F0E0017D6EC2CF033C182F40401300E74
:102DA000822773EC0EF0AFC500F101010F0E001782
:102DB000D6EC2CF033C182F40401300E822773EC80
:102DC0000EF0120084C3E8FF0F0BE83AE8CFB5F528
:102DD00085C3E8FF0F0B0501B51387C3E8FF0F0B91
:102DE000E83AE8CFB4F588C3E8FF0F0B0501B41348
:102DF0008AC3E8FF0F0BE83AE8CFB3F58BC3E8FFCF
:102E00000F0B0501B3138DC3E8FF0F0BE8CFB2F52D
:102E10008FC3E8FF0F0BE83AE8CFB1F590C3E8FFA6
:102E20000F0B0501B11392C3E8FF0F0BE83AE8CF8F
:102E3000B0F593C3E8FF0F0B0501B01395C3E8FF8E
:102E40000F0BE83AE8CFAFF596C3E8FF0F0B05018B
:102E5000AF1316EC2EF004014C0E826F73EC0EF0E3
:102E60000401430E826F73EC0EF0F4EF15F007844B
:102E700004014C0E826F73EC0EF00401370E826F6A
:102E800073EC0EF004012C0E826F73EC0EF0050152
:102E90002E51130A06E005012E51170A0DE0D2EF5C
:102EA00017F00101000E006F000E016F100E026F8F
:102EB000000E036F65EF17F00101000E006F000EAA
:102EC000016F000E026F010E036FD6EC2CF02AC1C9
:102ED00082F40401300E822773EC0EF02BC182F4D1
:102EE0000401300E822773EC0EF02CC182F4040131
:102EF000300E822773EC0EF02DC182F40401300EE7
:102F0000822773EC0EF02EC182F40401300E82276A
:102F100073EC0EF02FC182F40401300E822773ECA3
:102F20000EF030C182F40401300E822773EC0EF0F3
:102F300031C182F40401300E822773EC0EF032C1ED
:102F400082F40401300E822773EC0EF033C182F458
:102F50000401300E822773EC0EF004012C0E826FF8
:102F600073EC0EF00101100E006F000E016F000EE9
:102F7000026F000E036FD6EC2CF031C182F4040115
:102F8000300E822773EC0EF032C182F40401300E51
:102F9000822773EC0EF033C182F40401300E8227D5
:102FA00073EC0EF00794FCEF1CF00501216B226B13
:102FB000236B246B04014C0E826F73EC0EF0040142
:102FC000380E826F73EC0EF004012C0E826F73ECDE
:102FD0000EF00101100E006F000E016F000E026F67
:102FE000000E036FD6EC2CF02AC182F40401300EDF
:102FF000822773EC0EF02BC182F40401300E82277D
:1030000073EC0EF02CC182F40401300E822773ECB5
:103010000EF02DC182F40401300E822773EC0EF005
:103020002EC182F40401300E822773EC0EF02FC102
:1030300082F40401300E822773EC0EF030C182F46A
:103040000401300E822773EC0EF031C182F40401CA
:10305000300E822773EC0EF032C182F40401300E80
:10306000822773EC0EF033C182F40401300E822704
:1030700073EC0EF004012C0E826F73EC0EF025C57C
:1030800000F126C501F127C502F128C503F10101B0
:10309000100E046F000E056F000E066F000E076F16
:1030A00069EC2CF000C133F501C134F502C135F5EE
:1030B00003C136F5D6EC2CF02AC182F40401300E9F
:1030C000822773EC0EF02BC182F40401300E8227AC
:1030D00073EC0EF02CC182F40401300E822773ECE5
:1030E0000EF02DC182F40401300E822773EC0EF035
:1030F0002EC182F40401300E822773EC0EF02FC132
:1031000082F40401300E822773EC0EF030C182F499
:103110000401300E822773EC0EF031C182F40401F9
:10312000300E822773EC0EF032C182F40401300EAF
:10313000822773EC0EF033C182F40401300E822733
:1031400073EC0EF07DEC0EF005013367AFEF18F075
:103150003467AFEF18F03567AFEF18F0366702D07D
:103160004EEF19F0129E129C21C500F122C501F10B
:1031700023C502F124C503F1899A400EC76E200EC3
:10318000C66E9E96C69E0B0EC96EFF0E9EB602D0F0
:10319000E82EFCD79E96C69E02C1C9FFFF0E9EB6C2
:1031A00002D0E82EFCD79E96C69E01C1C9FFFF0E35
:1031B0009EB602D0E82EFCD79E96C69E00C1C9FFDF
:1031C000FF0E9EB602D0E82EFCD79E96C69EC95230
:1031D000FF0E9EB602D0E82EFCD70501100E326F0E
:1031E000040114EE00F080517F0BE1269E96C69EEE
:1031F000C952FF0E9EB602D0E82EFCD7C9CFE7FF1A
:103200000401802B0501322FF0EF18F0898A33C5B5
:1032100000F134C501F135C502F136C503F10101F4
:10322000010E046F000E056F000E066F000E076F93
:1032300038EC2CF000C133F501C134F502C135F58D
:1032400003C136F5050133672DEF19F034672DEF13
:1032500019F035672DEF19F0366702D04EEF19F0EF
:1032600021C500F122C501F123C502F124C503F1F6
:103270000101100E046F000E056F000E066F000EA8
:10328000076F3DEC2CF000C121F501C122F502C110
:1032900023F503C124F5128E57EF26F00401450EE5
:1032A000826F73EC0EF004014F0E826F73EC0EF020
:1032B0000401460E826F73EC0EF0FCEF1CF00784E5
:1032C000B4EC33F033EC2DF02DC500F1D6EC2CF03E
:1032D00004014C0E826F73EC0EF00401300E826F0D
:1032E00073EC0EF004012C0E826F73EC0EF031C102
:1032F00082F40401300E822773EC0EF032C182F4A6
:103300000401300E822773EC0EF033C182F4040105
:10331000300E822773EC0EF004012C0E826F73ECDA
:103320000EF033EC2DF02EC500F1D6EC2CF031C1AF
:1033300082F40401300E822773EC0EF032C182F465
:103340000401300E822773EC0EF033C182F40401C5
:10335000300E822773EC0EF00794FCEF1CF0040192
:103360004C0E826F73EC0EF00401650E826F73ECED
:103370000EF0D9EC2FF0FCEF1CF004014C0E826F24
:1033800073EC0EF00401450E826F73EC0EF0F0EC5E
:103390002FF0FCEF1CF004014C0E826F73EC0EF06A
:1033A0000401620E826F73EC0EF01EEC30F0FCEF45
:1033B0001CF004014C0E826F73EC0EF00401420EFF
:1033C000826F73EC0EF007EC30F0FCEF1CF00401A0
:1033D0004C0E826F73EC0EF00401760E826F73EC6C
:1033E0000EF004012C0E826F73EC0EF010A807D0C3
:1033F0000401310E826F73EC0EF0FCEF1CF004013F
:10340000300E826F73EC0EF0FCEF1CF004014C0EDA
:10341000826F73EC0EF004015A0E826F73EC0EF0A3
:1034200004012C0E826F73EC0EF0B4EC33F033EC2D
:103430002DF005012E51130A06E005012E51170A41
:103440000DE037EF1AF00101000E006F000E016F62
:10345000100E026F000E036F37EF1AF00101000E1D
:10346000006F000E016F000E026F010E036F01016D
:10347000100E046F000E056F000E066F000E076F32
:1034800069EC2CF0D6EC2CF02AC182F40401300E49
:10349000822773EC0EF02BC182F40401300E8227D8
:1034A00073EC0EF02CC182F40401300E822773EC11
:1034B0000EF02DC182F40401300E822773EC0EF061
:1034C0002EC182F40401300E822773EC0EF02FC15E
:1034D00082F40401300E822773EC0EF030C182F4C6
:1034E0000401300E822773EC0EF031C182F4040126
:1034F000300E822773EC0EF032C182F40401300EDC
:10350000822773EC0EF033C182F40401300E82275F
:1035100073EC0EF0FCEF1CF0078404014C0E826F7C
:1035200073EC0EF00401310E826F73EC0EF00401A7
:103530002C0E826F73EC0EF025C500F126C501F14B
:1035400027C502F128C503F10101100E046F000E1A
:10355000056F000E066F000E076F69EC2CF0D6ECBD
:103560002CF02AC182F40401300E822773EC0EF095
:103570002BC182F40401300E822773EC0EF02CC1B3
:1035800082F40401300E822773EC0EF02DC182F418
:103590000401300E822773EC0EF02EC182F4040178
:1035A000300E822773EC0EF02FC182F40401300E2E
:1035B000822773EC0EF030C182F40401300E8227B2
:1035C00073EC0EF031C182F40401300E822773ECEB
:1035D0000EF032C182F40401300E822773EC0EF03B
:1035E00033C182F40401300E822773EC0EF007948D
:1035F000FCEF1CF0078404014C0E826F73EC0EF09C
:103600000401320E826F73EC0EF00CEC32F0079472
:10361000FCEF1CF0078404014C0E826F73EC0EF07B
:103620000401330E826F73EC0EF069EC32F00794F4
:1036300097EF1AF0078404014C0E826F73EC0EF0C2
:103640000401340E826F73EC0EF004012C0E826FB5
:1036500073EC0EF074EC2DF084C32AF185C32BF1CA
:1036600086C32CF187C32DF188C32EF189C32FF1B6
:103670008AC330F18BC331F18CC332F18DC333F186
:103680000101296B81EC2DF0F8EC2CF0100E046F89
:10369000000E056F000E066F000E076F49EC2CF050
:1036A00000C121F501C122F502C123F503C124F5B2
:1036B00067EC33F038C5AFF539C5B0F53AC5B1F5AB
:1036C0003BC5B2F53CC5B3F53DC5B4F53EC5B5F552
:1036D000FFEC15F004012C0E826F73EC0EF03FC569
:1036E00000F140C501F141C502F142C503F10101FC
:1036F000000E046F000E056F010E066F000E076FBF
:1037000069EC2CF0D6EC2CF0296789EF1BF08EEFDA
:103710001BF004012D0E826F73EC0EF030C182F4A9
:103720000401300E822773EC0EF031C182F40401E3
:10373000300E822773EC0EF004012E0E826F73ECB4
:103740000EF032C182F40401300E822773EC0EF0C9
:1037500033C182F40401300E822773EC0EF00401B1
:103760002C0E826F73EC0EF033EC2DF043C500F19C
:1037700044C501F181EC27F004012C0E826F73EC3B
:103780000EF033EC2DF045C500F1D6EC2CF031C134
:1037900082F40401300E822773EC0EF032C182F401
:1037A0000401300E822773EC0EF033C182F4040161
:1037B000300E822773EC0EF004012C0E826F73EC36
:1037C0000EF037C5E8FFE8B806D00401300E826F6E
:1037D00073EC0EF005D00401310E826F73EC0EF025
:1037E0000794FCEF1CF074EC2DF085C32AF186C31E
:1037F0002BF187C32CF188C32DF189C32EF18AC325
:103800002FF18BC330F18CC331F18DC332F18EC3F4
:1038100033F10101296B81EC2DF0F8EC2CF0010162
:10382000010E046F000E056F000E066F000E076F8D
:1038300038EC2CF0100E046F000E056F000E066FB2
:10384000000E076F49EC2CF000C129F501C12AF5E3
:1038500002C12BF503C12CF593EC31F004014C0EA1
:10386000826F73EC0EF00401460E826F73EC0EF063
:1038700004012C0E826F73EC0EF025C500F126C5F5
:1038800001F127C502F128C503F10101100E046FF3
:10389000000E056F000E066F000E076F69EC2CF02E
:1038A000D6EC2CF02AC182F40401300E822773EC8E
:1038B0000EF02BC182F40401300E822773EC0EF05F
:1038C0002CC182F40401300E822773EC0EF02DC15E
:1038D00082F40401300E822773EC0EF02EC182F4C4
:1038E0000401300E822773EC0EF02FC182F4040124
:1038F000300E822773EC0EF030C182F40401300EDA
:10390000822773EC0EF031C182F40401300E82275D
:1039100073EC0EF032C182F40401300E822773EC96
:103920000EF033C182F40401300E822773EC0EF0E6
:10393000FCEF1CF00F9869EC32F0308057EF26F066
:1039400004014C0E826F73EC0EF00401350E826F91
:1039500073EC0EF004012C0E826F73EC0EF033EC5E
:103960002DF00784B9C500F10794D6EC2CF031C1D5
:1039700082F40401300E822773EC0EF032C182F41F
:103980000401300E822773EC0EF033C182F404017F
:10399000300E822773EC0EF0FCEF1CF02CEC32F0B2
:1039A00033EC2DF037C500F1D6EC2CF004014C0EB1
:1039B000826F73EC0EF00401360E826F73EC0EF022
:1039C00004012C0E826F73EC0EF031C182F40401FD
:1039D000300E822773EC0EF032C182F40401300EF7
:1039E000822773EC0EF033C182F40401300E82277B
:1039F00073EC0EF0FCEF1CF07DEC0EF057EF26F0B0
:103A000004014C0E826F73EC0EF00401500E826FB5
:103A100073EC0EF004012C0E826F73EC0EF085C374
:103A20002AF186C32BF187C32CF188C32DF189C3FA
:103A30002EF18AC32FF18BC330F18CC331F18DC3CA
:103A400032F18EC333F1010181EC2DF0F8EC2CF052
:103A500003018451530A0DE0030184514D0A38E0FB
:103A60000401780E826F73EC0EF07DEC0EF057EFD0
:103A700026F00401530E826F73EC0EF0250E0C6ECF
:103A800000C10BF00AEC0BF0260E0C6E01C10BF01E
:103A90000AEC0BF0270E0C6E02C10BF00AEC0BF0D7
:103AA000280E0C6E03C10BF00AEC0BF000C157F5A9
:103AB00001C158F502C159F503C15AF500C15BF5C2
:103AC00001C15CF502C15DF503C15EF5DDEF1DF0DE
:103AD00004014D0E826F73EC0EF0290E0C6E00C1C6
:103AE0000BF00AEC0BF000C15FF500C160F5DDEFF3
:103AF0001DF004014C0E826F73EC0EF00401540EA5
:103B0000826F73EC0EF004012C0E826F73EC0EF0DA
:103B100084C32AF185C32BF186C32CF187C32DF111
:103B200088C32EF189C32FF18AC330F18BC331F1E1
:103B30008DC332F18EC333F1010181EC2DF0F8EC2D
:103B40002CF00101000E046F000E056F010E066FD0
:103B5000000E076F49EC2CF0210E0C6E00C10BF02B
:103B60000AEC0BF0220E0C6E01C10BF00AEC0BF00C
:103B7000230E0C6E02C10BF00AEC0BF0240E0C6E3F
:103B800003C10BF00AEC0BF000C161F501C162F555
:103B900002C163F503C164F5DDEF1DF004014C0EB5
:103BA000826F73EC0EF00401490E826F73EC0EF01D
:103BB00004012C0E826F73EC0EF0250E21EC0BF03D
:103BC000E8CF00F1260E21EC0BF0E8CF01F1270E33
:103BD00021EC0BF0E8CF02F1280E21EC0BF0E8CF3E
:103BE00003F1D6EC2CF099EC2AF00401730E826FED
:103BF00073EC0EF004012C0E826F73EC0EF033ECBC
:103C00002DF0290E21EC0BF0E8CF00F1D6EC2CF0D2
:103C100099EC2AF004016D0E826F73EC0EF0040132
:103C20002C0E826F73EC0EF05BC500F15CC501F1E8
:103C30005DC502F15EC503F1D6EC2CF099EC2AF0DB
:103C40000401730E826F73EC0EF004012C0E826F70
:103C500073EC0EF033EC2DF060C500F1D6EC2CF0D7
:103C600099EC2AF004016D0E826F73EC0EF00401E2
:103C70002C0E826F73EC0EF061C500F162C501F18C
:103C800063C502F164C503F172EC26F004012C0E49
:103C9000826F73EC0EF07DEC0EF057EF26F083C3CD
:103CA0002AF184C32BF185C32CF186C32DF187C380
:103CB0002EF188C32FF189C330F18AC331F18BC350
:103CC00032F18CC333F1010181EC2DF0F8EC2CF0D2
:103CD000160E0C6E00C10BF00AEC0BF0170E0C6EFA
:103CE00001C10BF00AEC0BF0180E0C6E02C10BF0C8
:103CF0000AEC0BF0190E0C6E03C10BF00AEC0BF082
:103D000000C18AF101C18BF102C18CF103C18DF1B7
:103D100000C18EF101C18FF102C190F103C191F197
:103D200031EF1FF083C32AF184C32BF185C32CF13B
:103D300086C32DF187C32EF188C32FF189C330F1DB
:103D40008AC331F18BC332F18CC333F1010181ECB1
:103D50002DF0F8EC2CF000C18AF101C18BF102C109
:103D60008CF103C18DF100C18EF101C18FF102C14F
:103D700090F103C191F131EF1FF083C32AF184C3A5
:103D80002BF185C32CF186C32DF187C32EF188C397
:103D90002FF189C330F18AC331F18CC332F18DC365
:103DA00033F1010181EC2DF0F8EC2CF00101000E53
:103DB000046F000E056F010E066F000E076F49ECD1
:103DC0002CF01A0E0C6E00C10BF00AEC0BF01B0E5F
:103DD0000C6E01C10BF00AEC0BF01C0E0C6E02C154
:103DE0000BF00AEC0BF01D0E0C6E03C10BF00AEC8D
:103DF0000BF000C192F101C193F102C194F103C132
:103E000095F131EF1FF083C32AF184C32BF185C3F1
:103E10002CF186C32DF187C32EF188C32FF189C3FE
:103E200030F18AC331F18CC332F18DC333F101011A
:103E300081EC2DF0F8EC2CF00101000E046F000E67
:103E4000056F010E066F000E076F49EC2CF000C1E4
:103E500092F101C193F102C194F103C195F131EFE7
:103E60001FF0160E21EC0BF0E8CF00F1170E21EC3D
:103E70000BF0E8CF01F1180E21EC0BF0E8CF02F1C6
:103E8000190E21EC0BF0E8CF03F1D6EC2CF099ECF5
:103E90002AF00401730E826F73EC0EF004012C0EF5
:103EA000826F73EC0EF08AC100F18BC101F18CC1FD
:103EB00002F18DC103F1D6EC2CF099EC2AF004014B
:103EC000730E826F73EC0EF004012C0E826F73EC94
:103ED0000EF01A0E21EC0BF0E8CF00F11B0E21ECD6
:103EE0000BF0E8CF01F11C0E21EC0BF0E8CF02F152
:103EF0001D0E21EC0BF0E8CF03F172EC26F004016B
:103F00002C0E826F73EC0EF092C100F193C101F19F
:103F100094C102F195C103F172EC26F07DEC0EF034
:103F200057EF26F00401690E826F73EC0EF0040166
:103F30002C0E826F73EC0EF00101040E006F000E68
:103F4000016F000E026F000E036FD6EC2CF02CC137
:103F500082F40401300E822773EC0EF02DC182F43E
:103F60000401300E822773EC0EF02EC182F404019E
:103F7000300E822773EC0EF02FC182F40401300E54
:103F8000822773EC0EF030C182F40401300E8227D8
:103F900073EC0EF031C182F40401300E822773EC11
:103FA0000EF032C182F40401300E822773EC0EF061
:103FB00033C182F40401300E822773EC0EF0040149
:103FC0002C0E826F73EC0EF00101060E006F000ED6
:103FD000016F000E026F000E036FD6EC2CF02CC1A7
:103FE00082F40401300E822773EC0EF02DC182F4AE
:103FF0000401300E822773EC0EF02EC182F404010E
:10400000300E822773EC0EF02FC182F40401300EC3
:10401000822773EC0EF030C182F40401300E822747
:1040200073EC0EF031C182F40401300E822773EC80
:104030000EF032C182F40401300E822773EC0EF0D0
:1040400033C182F40401300E822773EC0EF00401B8
:104050002C0E826F73EC0EF00101360E006F000E15
:10406000016F000E026F000E036FD6EC2CF02CC116
:1040700082F40401300E822773EC0EF02DC182F41D
:104080000401300E822773EC0EF02EC182F404017D
:10409000300E822773EC0EF02FC182F40401300E33
:1040A000822773EC0EF030C182F40401300E8227B7
:1040B00073EC0EF031C182F40401300E822773ECF0
:1040C0000EF032C182F40401300E822773EC0EF040
:1040D00033C182F40401300E822773EC0EF0040128
:1040E0002C0E826F73EC0EF0200EF86EF76AF66AF3
:1040F00004010900F5CF82F473EC0EF00900F5CF4E
:1041000082F473EC0EF00900F5CF82F473EC0EF03C
:104110000900F5CF82F473EC0EF00900F5CF82F4BC
:1041200073EC0EF00900F5CF82F473EC0EF0090089
:10413000F5CF82F473EC0EF00900F5CF82F473EC46
:104140000EF07DEC0EF057EF26F08351630AD8A4F1
:1041500055EF26F08451610AD8A455EF26F0855119
:104160006C0AD8A455EF26F08651410A3FE08651EB
:10417000440A1BE08651420AD8B409EF21F0865167
:10418000350AD8B4E1EF27F08651360AD8B436EFB5
:1041900028F08651370AD8B49FEF28F08651380AA4
:1041A000D8B4FDEF28F055EF26F00798079A0401E0
:1041B0007A0E826F73EC0EF00401780E826F73EC4E
:1041C0000EF00401640E826F73EC0EF00401550EC4
:1041D000826F73EC0EF0F2EF20F004014C0E826F50
:1041E00073EC0EF07DEC0EF057EF26F00788079A7F
:1041F00004017A0E826F73EC0EF00401410E826F9F
:1042000073EC0EF00401610E826F73EC0EF0E6EFBA
:1042100020F00798078A04017A0E826F73EC0EF083
:104220000401420E826F73EC0EF00401610E826F86
:1042300073EC0EF0E6EF20F00101666727EF21F046
:10424000676727EF21F0686727EF21F0696715D0CE
:104250004F6732EF21F0506732EF21F0516732EFB4
:1042600021F052670AD00101000E006F000E016FAD
:10427000000E026F000E036F120011B80AD0010188
:10428000620E046F010E056F000E066F000E076FC1
:1042900009D00101A70E046F020E056F000E066F14
:1042A000000E076F66C100F167C101F168C102F13C
:1042B00069C103F138EC2CF003BFCFEF21F0119A64
:1042C000119C0101000E046FA80E056F550E066FBC
:1042D000020E076F66C100F167C101F168C102F10A
:1042E00069C103F166C186F167C187F168C188F1D0
:1042F00069C189F138EC2CF003BF0BD00101000E2D
:10430000866FA80E876F550E886F020E896F118A0F
:10431000119C0E0E21EC0BF0E8CF18F10F0E21ECE2
:104320000BF0E8CF19F1100E21EC0BF0E8CF1AF1E9
:10433000110E21EC0BF0E8CF1BF181EC2BF086C1C4
:1043400004F187C105F188C106F189C107F138EC94
:104350002CF0078245EC2BF081EC2BF0079245EC1A
:104360002BF086C100F187C101F188C102F189C13A
:1043700003F1079245EC2BF0CC0E046FE00E056FB5
:10438000870E066F050E076F38EC2CF000C118F190
:1043900001C119F102C11AF103C11BF13BD0119CFB
:1043A000119A0101800E006F1A0E016F060E026F46
:1043B000000E036F4FC104F150C105F151C106F168
:1043C00052C107F138EC2CF003AF05D033EC2DF0DF
:1043D000118C119A12000E0E21EC0BF0E8CF18F19F
:1043E0000F0E21EC0BF0E8CF19F1100E21EC0BF0C1
:1043F000E8CF1AF1110E21EC0BF0E8CF1BF14FC101
:1044000000F150C101F151C102F152C103F1078223
:1044100045EC2BF018C100F119C101F11AC102F1EC
:104420001BC103F112000401730E826F73EC0EF0D6
:1044300004012C0E826F73EC0EF0078462C166F1EA
:1044400063C167F164C168F165C169F14BC14FF1A6
:104450004CC150F14DC151F14EC152F157C159F10A
:1044600058C15AF1079439EC22F07DEC0EF057EF69
:1044700026F066C100F167C101F168C102F169C1AE
:1044800003F10101D6EC2CF099EC2AF00401630E43
:10449000826F73EC0EF004012C0E826F73EC0EF041
:1044A0004FC100F150C101F151C102F152C103F1FC
:1044B0000101D6EC2CF099EC2AF00401660E826F13
:1044C00073EC0EF004012C0E826F73EC0EF033ECE3
:1044D0002DF059C100F15AC101F10101D6EC2CF0C7
:1044E00099EC2AF00401740E826F73EC0EF0120046
:1044F00010820401530E826F73EC0EF004012C0E37
:10450000826F73EC0EF083C32AF184C32BF185C351
:104510002CF186C32DF187C32EF188C32FF189C3F7
:1045200030F18AC331F18BC332F18CC333F1010115
:1045300081EC2DF0F8EC2CF000C166F101C167F1BF
:1045400002C168F103C169F18EC32AF18FC32BF157
:1045500090C32CF191C32DF192C32EF193C32FF18F
:1045600094C330F195C331F196C332F197C333F15F
:10457000010181EC2DF0F8EC2CF000C14FF101C1EC
:1045800050F102C151F103C152F174EC2DF099C305
:104590002FF19AC330F19BC331F19CC332F19DC31B
:1045A00033F1010181EC2DF0F8EC2CF000C159F150
:1045B00001C15AF139EC22F004012C0E826F73EC28
:1045C0000EF0F2EF22F0118E19A002D019AE108C6D
:1045D00018BE02D018A4108E8251520A02E10F8236
:1045E00001D00F928251750A02E1108401D010941B
:1045F0008251550A02E1108601D0109611A003D015
:1046000011A401D01084078410B260EF23F010A42D
:104610004CEF23F0B6C166F1B7C167F1B8C168F1DC
:10462000B9C169F1BAC16AF1BBC16BF1BCC16CF12E
:10463000BDC16DF1BEC16EF1BFC16FF1C0C170F1FE
:10464000C1C171F1C2C172F1C3C173F1C4C174F1CE
:10465000C5C175F1C6C176F1C7C177F1C8C178F19E
:10466000C9C179F1CAC17AF1CBC17BF1CCC17CF16E
:10467000CDC17DF1CEC17EF1CFC17FF1D0C180F13E
:10468000D1C181F1D2C182F1D3C183F1D4C184F10E
:10469000D5C185F154EF23F062C166F163C167F1C2
:1046A00064C168F165C169F14BC14FF14CC150F172
:1046B0004DC151F14EC152F157C159F158C15AF192
:1046C00007940FA082EF23F0010192676FEF23F0B0
:1046D00093676FEF23F094676FEF23F0956773EFA5
:1046E00023F082EF23F01CEC21F092C104F193C17E
:1046F00005F194C106F195C107F138EC2CF003BF28
:104700001DEF26F01CEC21F00101000E046F000EDD
:10471000056F010E066F000E076F69EC2CF011A0FB
:104720002AD011A228D0D6EC2CF0296701D005D0D0
:1047300004012D0E826F73EC0EF030C182F404017F
:10474000300E822773EC0EF031C182F40401300E7A
:10475000822773EC0EF032C182F40401300E8227FE
:1047600073EC0EF033C182F40401300E822773EC37
:104770000EF07DEC0EF012A8C3D012981AC01BF0F8
:104780001B3A1B42070E1B1600011B50000AD8B42F
:104790004EEF24F000011B50010AD8B4DAEF23F0E9
:1047A00000011B50020AD8B4D8EF23F080EF24F0A8
:1047B00080EF24F033EC2DF02AC001F12BC000F182
:1047C000D89001330033D890013300330101630ED8
:1047D000046F000E056F000E066F000E076F69EC88
:1047E0002CF0280E046F000E056F000E066F000EF1
:1047F000076F38EC2CF000C12DF033EC2DF028C001
:1048000001F1019F019D29C000F10101A40E046F77
:10481000000E056F000E066F000E076F69EC2CF09E
:1048200000C12CF000C104F101C105F102C106F183
:1048300003C107F1640E006F000E016F000E026FDE
:10484000000E036F38EC2CF0050E046F000E056FA0
:10485000000E066F000E076F69EC2CF000C104F12A
:1048600001C105F102C106F103C107F133EC2DF0DE
:104870002DC000F138EC2CF000C12EF02EC0E8FF66
:10488000050F2D5C03E78A8480EF24F02EC0E8FF3B
:104890000A0F2D5C01E68A9480EF24F000C124F118
:1048A00001C125F102C126F103C127F133EC2DF03E
:1048B00039EC2DF01A501F0BE8CF00F10101640E06
:1048C000046F000E056F000E066F000E076F49ECB7
:1048D0002CF024C104F125C105F126C106F127C140
:1048E00007F138EC2CF003BF02D08A9401D08A84FF
:1048F00024C100F125C101F126C102F127C103F154
:1049000000C124F101C125F102C126F103C127F143
:1049100010AE4DD0109E00C108F101C109F102C1D5
:104920000AF103C10BF1D6EC2CF030C1D6F131C144
:10493000D7F132C1D8F133C1D9F108C100F109C1B1
:1049400001F10AC102F10BC103F101016C0E046F08
:10495000070E056F000E066F000E076F38EC2CF087
:1049600003BF04D00101550EDA6F1CD008C100F15D
:1049700009C101F10AC102F10BC103F10101A40E49
:10498000046F060E056F000E066F000E076F38EC01
:104990002CF003BF04D001017F0EDA6F03D00101B8
:1049A000FF0EDA6F1C8E11AE1DEF26F0119E24C192
:1049B00000F125C101F126C102F127C103F111A0C7
:1049C00005D011A203D00FB01DEF26F010A4F0EF18
:1049D00024F00401750E826F73EC0EF0F5EF24F0F5
:1049E0000401720E826F73EC0EF004012C0E826FC4
:1049F00073EC0EF0D6EC2CF0296704EF25F00401DF
:104A0000200E826F07EF25F004012D0E826F73ECEC
:104A10000EF030C182F40401300E822773EC0EF0E8
:104A200031C182F40401300E822773EC0EF00401D0
:104A30002E0E826F73EC0EF032C182F40401300E40
:104A4000822773EC0EF033C182F40401300E82270A
:104A500073EC0EF004016D0E826F73EC0EF0040126
:104A60002C0E826F73EC0EF04FC100F150C101F1BA
:104A700051C102F152C103F10101D6EC2CF099ECC5
:104A80002AF00401480E826F73EC0EF004017A0ED6
:104A9000826F73EC0EF004012C0E826F73EC0EF03B
:104AA00066C100F167C101F168C102F169C103F19A
:104AB0000101D6EC2CF099EC2AF00401630E826F10
:104AC00073EC0EF004012C0E826F73EC0EF066C1D5
:104AD00000F167C101F168C102F169C103F101018F
:104AE0000A0E046F000E056F000E066F000E076FB2
:104AF00049EC2CF0000E046F120E056F000E066FCD
:104B0000000E076F69EC2CF0D6EC2CF02AC182F471
:104B10000401300E822773EC0EF02BC182F40401E5
:104B2000300E822773EC0EF02CC182F40401300E9B
:104B3000822773EC0EF02DC182F40401300E82271F
:104B400073EC0EF02EC182F40401300E822773EC58
:104B50000EF02FC182F40401300E822773EC0EF0A8
:104B600030C182F40401300E822773EC0EF0040190
:104B70002E0E826F73EC0EF031C182F40401300E00
:104B8000822773EC0EF032C182F40401300E8227CA
:104B900073EC0EF033C182F40401300E822773EC03
:104BA0000EF00401730E826F73EC0EF004012C0EF4
:104BB000826F73EC0EF033EC2DF059C100F15AC145
:104BC00001F181EC27F00FB2E9EF25F00FA01BEF08
:104BD00026F004012C0E826F73EC0EF0200EF86E9E
:104BE000F76AF66A04010900F5CF82F473EC0EF05F
:104BF0000900F5CF82F473EC0EF00900F5CF82F4D2
:104C000073EC0EF00900F5CF82F473EC0EF009009E
:104C1000F5CF82F473EC0EF00900F5CF82F473EC5B
:104C20000EF00900F5CF82F473EC0EF00900F5CF19
:104C300082F473EC0EF07DEC0EF00F9057EF26F03F
:104C40000401630E826F73EC0EF004012C0E826F70
:104C500073EC0EF05DEC26F004012C0E826F73EC09
:104C60000EF0D0EC26F004012C0E826F73EC0EF0E7
:104C70004CEC27F004012C0E826F73EC0EF0010156
:104C8000F80E006FCD0E016F660E026F030E036FFC
:104C900072EC26F004012C0E826F73EC0EF062ECC5
:104CA00027F07DEC0EF057EF26F07DEC0EF00301BF
:104CB000C26B0790109266EF29F0D8900E0E21EC8F
:104CC0000BF0E8CF00F10F0E21EC0BF0E8CF01F173
:104CD000100E21EC0BF0E8CF02F1110E21EC0BF0DD
:104CE000E8CF03F10101000E046F000E056F010E05
:104CF000066F000E076F69EC2CF0D6EC2CF02AC181
:104D000082F40401300E822773EC0EF02BC182F482
:104D10000401300E822773EC0EF02CC182F40401E2
:104D2000300E822773EC0EF02DC182F40401300E98
:104D3000822773EC0EF02EC182F40401300E82271C
:104D400073EC0EF02FC182F40401300E822773EC55
:104D50000EF030C182F40401300E822773EC0EF0A5
:104D600031C182F40401300E822773EC0EF004018D
:104D70002E0E826F73EC0EF032C182F40401300EFD
:104D8000822773EC0EF033C182F40401300E8227C7
:104D900073EC0EF004016D0E826F73EC0EF01200D6
:104DA000120E21EC0BF0E8CF00F1130E21EC0BF00A
:104DB000E8CF01F1140E21EC0BF0E8CF02F1150E53
:104DC00021EC0BF0E8CF03F101010A0E046F000E95
:104DD000056F000E066F000E076F49EC2CF0000EF9
:104DE000046F120E056F000E066F000E076F69EC60
:104DF0002CF0D6EC2CF02AC182F40401300E82276C
:104E000073EC0EF02BC182F40401300E822773EC98
:104E10000EF02CC182F40401300E822773EC0EF0E8
:104E20002DC182F40401300E822773EC0EF02EC1E6
:104E300082F40401300E822773EC0EF02FC182F44D
:104E40000401300E822773EC0EF030C182F40401AD
:104E5000300E822773EC0EF004012E0E826F73EC7D
:104E60000EF031C182F40401300E822773EC0EF093
:104E700032C182F40401300E822773EC0EF033C18C
:104E800082F40401300E822773EC0EF00401730EDD
:104E9000826F73EC0EF012000A0E21EC0BF0E8CFDB
:104EA00000F10B0E21EC0BF0E8CF01F10C0E21EC20
:104EB0000BF0E8CF02F10D0E21EC0BF0E8CF03F17F
:104EC00081EF27F0060E21EC0BF0E8CF00F1070E82
:104ED00021EC0BF0E8CF01F1080E21EC0BF0E8CF4C
:104EE00002F1090E21EC0BF0E8CF03F181EF27F07E
:104EF000010133EC2DF0078457C100F158C101F1D5
:104F000007940101E80E046F800E056F000E066F16
:104F1000000E076F49EC2CF0000E046F040E056FB5
:104F2000000E066F000E076F69EC2CF0880E046F00
:104F3000130E056F000E066F000E076F38EC2CF095
:104F40000A0E046F000E056F000E066F000E076F4D
:104F500069EC2CF0D6EC2CF001012967B5EF27F0B5
:104F60000401200E826FB8EF27F004012D0E826F2E
:104F700073EC0EF030C182F40401300E822773EC22
:104F80000EF031C182F40401300E822773EC0EF072
:104F900032C182F40401300E822773EC0EF004015A
:104FA0002E0E826F73EC0EF033C182F40401300ECA
:104FB000822773EC0EF00401430E826F73EC0EF047
:104FC000120087C32AF188C32BF189C32CF18AC34D
:104FD0002DF18BC32EF18CC32FF18DC330F18EC315
:104FE00031F190C332F191C333F10101296B81ECAE
:104FF0002DF0F8EC2CF00101000E046F000E056F8F
:10500000010E066F000E076F49EC2CF00E0E0C6EB1
:1050100000C10BF00AEC0BF00F0E0C6E01C10BF08F
:105020000AEC0BF0100E0C6E02C10BF00AEC0BF048
:10503000110E0C6E03C10BF00AEC0BF004017A0E9A
:10504000826F73EC0EF004012C0E826F73EC0EF085
:105050000401350E826F73EC0EF004012C0E826F8A
:1050600073EC0EF05DEC26F0F2EF20F087C32AF12E
:1050700088C32BF189C32CF18AC32DF18BC32EF188
:105080008CC32FF18DC330F18EC331F190C332F157
:1050900091C333F10101296B81EC2DF0F8EC2CF078
:1050A000880E046F130E056F000E066F000E076F5B
:1050B0003DEC2CF0000E046F040E056F000E066F21
:1050C000000E076F49EC2CF00101E80E046F800E12
:1050D000056F000E066F000E076F69EC2CF00A0ECC
:1050E0000C6E00C10BF00AEC0BF00B0E0C6E01C144
:1050F0000BF00AEC0BF00C0E0C6E02C10BF00AEC7C
:105100000BF00D0E0C6E03C10BF00AEC0BF004015A
:105110007A0E826F73EC0EF004012C0E826F73EC2A
:105120000EF00401360E826F73EC0EF004012C0EAB
:10513000826F73EC0EF04CEC27F0F2EF20F087C397
:105140002AF188C32BF189C32CF18AC32DF18BC3BB
:105150002EF18CC32FF18DC330F18FC331F190C389
:1051600032F191C333F1010181EC2DF0F8EC2CF018
:10517000000E046F120E056F000E066F000E076F13
:1051800049EC2CF001010A0E046F000E056F000EB1
:10519000066F000E076F69EC2CF0120E0C6E00C14A
:1051A0000BF00AEC0BF0130E0C6E01C10BF00AECC5
:1051B0000BF0140E0C6E02C10BF00AEC0BF0150E86
:1051C0000C6E03C10BF00AEC0BF004017A0E826F37
:1051D00073EC0EF004012C0E826F73EC0EF00401E0
:1051E000370E826F73EC0EF004012C0E826F73EC9D
:1051F0000EF0D0EC26F0F2EF20F087C32AF188C33E
:105200002BF189C32CF18AC32DF18BC32EF18CC3F2
:105210002FF18DC330F18EC331F190C332F191C3C0
:1052200033F10101296B81EC2DF0F8EC2CF0880EA4
:10523000046F130E056F000E066F000E076F3DEC36
:105240002CF0000E046F040E056F000E066F000EAA
:10525000076F49EC2CF00101E80E046F800E056F1A
:10526000000E066F000E076F69EC2CF0060E0C6E38
:1052700000C10BF00AEC0BF0070E0C6E01C10BF035
:105280000AEC0BF0080E0C6E02C10BF00AEC0BF0EE
:10529000090E0C6E03C10BF00AEC0BF004017A0E40
:1052A000826F73EC0EF004012C0E826F73EC0EF023
:1052B0000401380E826F73EC0EF004012C0E826F25
:1052C00073EC0EF062EC27F0F2EF20F007A8D9EFB4
:1052D00029F00101800E006F1A0E016F060E026F99
:1052E000000E036F4BC104F14CC105F14DC106F135
:1052F0004EC107F138EC2CF003BF1FEF2AF093ECFE
:105300002AF04BC100F14CC101F14DC102F14EC177
:1053100003F1078245EC2BF018C104F119C105F126
:105320001AC106F11BC107F1F80E006FCD0E016F17
:10533000660E026F030E036F38EC2CF00E0E0C6E2F
:1053400000C10BF00AEC0BF00F0E0C6E01C10BF05C
:105350000AEC0BF0100E0C6E02C10BF00AEC0BF015
:10536000110E0C6E03C10BF00AEC0BF00784010167
:1053700033EC2DF057C100F158C101F107940A0E2A
:105380000C6E00C10BF00AEC0BF00B0E0C6E01C1A1
:105390000BF00AEC0BF00C0E0C6E02C10BF00AECD9
:1053A0000BF00D0E0C6E03C10BF00AEC0BF01FEFAF
:1053B0002AF007AA1FEF2AF00784010133EC2DF031
:1053C00057C100F158C101F10794060E0C6E00C1DF
:1053D0000BF00AEC0BF0070E0C6E01C10BF00AEC9F
:1053E0000BF0080E0C6E02C10BF00AEC0BF0090E6C
:1053F0000C6E03C10BF00AEC0BF0078462C100F1E4
:1054000063C101F164C102F165C103F10794120E99
:105410000C6E00C10BF00AEC0BF0130E0C6E01C108
:105420000BF00AEC0BF0140E0C6E02C10BF00AEC40
:105430000BF0150E0C6E03C10BF00AEC0BF0079885
:10544000079A0401805181197F0B0DE09EA8FED7B9
:1054500014EE00F081517F0BE126E750812B0F0104
:10546000AD6E21EF2AF005012F51010A13E081AA48
:105470005BEF2AF005012F51000A0AE00FB84AEF4E
:105480002AF0050130674AEF2AF00FB84AEF2AF0F8
:10549000F3EF33F081B85BEF2AF063EC2EF05BEFB3
:1054A0002AF0602F5BEF2AF05FC560F50501010E61
:1054B000306F3C0E316FBAEF0DF018C100F119C119
:1054C00001F11AC102F11BC103F1000E046F000EBD
:1054D000056F010E066F000E076F69EC2CF029A115
:1054E00088EF2AF02051D8B488EF2AF018C100F1D3
:1054F00019C101F11AC102F11BC103F1000E046FC1
:10550000000E056F0A0E066F000E076F69EC2CF097
:105510001200010104510013055101130651021339
:105520000751031312000101186B196B1A6B1B6BE7
:1055300012002AC182F40401300E822773EC0EF0AF
:105540002BC182F40401300E822773EC0EF02CC1C3
:1055500082F40401300E822773EC0EF02DC182F428
:105560000401300E822773EC0EF02EC182F4040188
:10557000300E822773EC0EF02FC182F40401300E3E
:10558000822773EC0EF030C182F40401300E8227C2
:1055900073EC0EF031C182F40401300E822773ECFB
:1055A0000EF032C182F40401300E822773EC0EF04B
:1055B00033C182F40401300E822773EC0EF0120026
:1055C0002FC182F40401300E822773EC0EF030C13B
:1055D00082F40401300E822773EC0EF031C182F4A4
:1055E0000401300E822773EC0EF032C182F4040104
:1055F000300E822773EC0EF033C182F40401300EBA
:10560000822773EC0EF01200060E1E6E060E1F6E41
:10561000060E206E1E2E0AEF2BF01F2E0AEF2BF027
:10562000202E0AEF2BF08B84020E1E6E020E1F6ED0
:10563000020E206E1E2E1AEF2BF01F2E1AEF2BF0EB
:10564000202E1AEF2BF08B941200FF0E1F6E1FC03E
:1056500020F0030E1E6E8B841E2E2BEF2BF0030EFC
:105660001E6E202E2BEF2BF08B941FC020F0030E0C
:105670001E6E1E2E39EF2BF0030E1E6E203E39EFEC
:105680002BF01F2E27EF2BF012000101005305E134
:10569000015303E1025301E1002B08EC2CF033EC41
:1056A0002DF03951006F3A51016F420E046F4B0ECD
:1056B000056F000E066F000E076F49EC2CF000C15D
:1056C00004F101C105F102C106F103C107F118C1DE
:1056D00000F119C101F11AC102F11BC103F107B2B6
:1056E00076EF2BF03DEC2CF078EF2BF038EC2CF033
:1056F00000C118F101C119F102C11AF103C11BF176
:10570000120033EC2DF059C100F15AC101F1060E1F
:1057100021EC0BF0E8CF04F1070E21EC0BF0E8CF01
:1057200005F1080E21EC0BF0E8CF06F1090E21EC93
:105730000BF0E8CF07F138EC2CF000C124F101C1E7
:1057400025F102C126F103C127F1290E046F000ED5
:10575000056F000E066F000E076F49EC2CF0EE0E81
:10576000046F430E056F000E066F000E076F3DECD1
:105770002CF024C104F125C105F126C106F127C191
:1057800007F149EC2CF000C11CF101C11DF102C16F
:105790001EF103C11FF1120E21EC0BF0E8CF04F152
:1057A000130E21EC0BF0E8CF05F1140E21EC0BF0F9
:1057B000E8CF06F1150E21EC0BF0E8CF07F10D0E46
:1057C000006F000E016F000E026F000E036F49ECB8
:1057D0002CF0180E046F000E056F000E066F000E01
:1057E000076F69EC2CF01CC104F11DC105F11EC14D
:1057F00006F11FC107F13DEC2CF06A0E046F2A0E72
:10580000056F000E066F000E076F38EC2CF01200CB
:10581000BF0EFA6E200E3A6F396BD8900037013701
:1058200002370337D8B019EF2CF03A2F0EEF2CF0D7
:1058300039073A070353D8B412000331070B800924
:105840003F6F03390F0B010F396F80EC5FF0406F32
:10585000390580EC5FF0405D405F396B3F33D8B075
:10586000392739333FA92EEF2CF040513927120048
:10587000010158EC2DF0D8B01200010103510719B5
:10588000346F1BEC2DF0D8900751031934AF800F03
:1058900012000101346B3FEC2DF0D8A055EC2DF037
:1058A000D8B012002AEC2DF033EC2DF01F0E366F1D
:1058B0006BEC2DF00B35D8B01BEC2DF0D8A00335D8
:1058C000D8B01200362F58EF2CF034B142EC2DF046
:1058D00012000101346B0451051106110711000873
:1058E000D8A03FEC2DF0D8A055EC2DF0D8B0120088
:1058F000086B096B0A6B0B6B6BEC2DF01F0E366F90
:105900006BEC2DF007510B5DD8A493EF2CF00651F2
:105910000A5DD8A493EF2CF00551095DD8A493EF4C
:105920002CF00451085DD8A0A6EF2CF00451085FBC
:105930000551D8A0053D095F0651D8A0063D0A5F74
:105940000751D8A0073D0B5FD8900081362F80EF1C
:105950002CF034B142EC2DF0346B3FEC2DF0D890AC
:105960006FEC2DF007510B5DD8A4C3EF2CF006515E
:105970000A5DD8A4C3EF2CF00551095DD8A4C3EF8C
:105980002CF00451085DD8A0D2EF2CF0003FD2EFEC
:105990002CF0013FD2EF2CF0023FD2EF2CF0032B82
:1059A000D8B4120034B142EC2DF012000101346B76
:1059B0003FEC2DF0D8B0120074EC2DF0200E366FB5
:1059C000003701370237033711EE33F00A0E376F15
:1059D000E7360A0EE75CD8B0E76EE552372FE8EFFE
:1059E0002CF0362FE0EF2CF034B12981D890120042
:1059F00001010A0E346F200E366F11EE29F034517A
:105A0000376F0A0ED890E652D8B0E726E732372F24
:105A100003EF2DF00333023301330033362FFDEF54
:105A20002CF0E750FF0FD8A00335D8B0120029B1F1
:105A300042EC2DF01200045100270551D8B0053D6D
:105A400001270651D8B0063D02270751D8B0073DBF
:105A5000032712000051086F0151096F02510A6FAC
:105A600003510B6F12000101006B016B026B036BA2
:105A700012000101046B056B066B076B1200033506
:105A8000D8A012000351800B001F011F021F031F2B
:105A9000003F52EF2DF0013F52EF2DF0023F52EF49
:105AA0002DF0032B342B032512000735D8A012004C
:105AB0000751800B041F051F061F071F043F68EFD7
:105AC0002DF0053F68EF2DF0063F68EF2DF0072B16
:105AD000342B072512000037013702370337083708
:105AE00009370A370B3712000101296B2A6B2B6B20
:105AF0002C6B2D6B2E6B2F6B306B316B326B336BD2
:105B0000120001012A510F0B2A6F2B510F0B2B6F23
:105B10002C510F0B2C6F2D510F0B2D6F2E510F0B86
:105B20002E6F2F510F0B2F6F30510F0B306F3151E4
:105B30000F0B316F32510F0B326F33510F0B336F2D
:105B4000120010A806D08994000EC76E220EC66EF1
:105B500005D08984000EC76E220EC66E050EE82E93
:105B6000FED7120010A802D0898401D08994050EB6
:105B7000E82EFED71200A1EC2DF09E96C69E000ED8
:105B8000C96EFF0E9EB602D0E82EFCD79E96C69E2A
:105B9000000EC96EFF0E9EB602D0E82EFCD7C9CF0C
:105BA000AFF59E96C69E000EC96EFF0E9EB602D041
:105BB000E82EFCD7C9CFB0F59E96C69E000EC96EE2
:105BC000FF0E9EB602D0E82EFCD7C9CFB1F59E9647
:105BD000C69E000EC96EFF0E9EB602D0E82EFCD700
:105BE000C9CFB2F59E96C69E000EC96EFF0E9EB638
:105BF00002D0E82EFCD7C9CFB3F59E96C69E000E04
:105C0000C96EFF0E9EB602D0E82EFCD7C9CFB4F500
:105C10009E96C69E000EC96EFF0E9EB602D0E82E5E
:105C2000FCD7C9CFB5F5B2EC2DF01200A1EC2DF0E8
:105C30009E96C69E800EC96EFF0E9EB602D0E82EBE
:105C4000FCD79E96C69EAFC5C9FFFF0E9EB602D07A
:105C5000E82EFCD79E96C69EB0C5C9FFFF0E9EB625
:105C600002D0E82EFCD79E96C69EB1C5C9FFFF0E96
:105C70009EB602D0E82EFCD79E96C69EB2C5C9FF3E
:105C8000FF0E9EB602D0E82EFCD79E96C69EB3C5E8
:105C9000C9FFFF0E9EB602D0E82EFCD79E96C69E88
:105CA000B4C5C9FFFF0E9EB602D0E82EFCD79E9663
:105CB000C69EB5C5C9FFFF0E9EB602D0E82EFCD722
:105CC000B2EC2DF01200A1EC2DF09E96C69E070EB0
:105CD000C96EFF0E9EB602D0E82EFCD79E96C69ED9
:105CE000000EC96EFF0E9EB602D0E82EFCD7C9CFBB
:105CF000AFF59E96C69E000EC96EFF0E9EB602D0F0
:105D0000E82EFCD7C9CFB0F59E96C69E000EC96E90
:105D1000FF0E9EB602D0E82EFCD7C9CFB1F59E96F5
:105D2000C69E000EC96EFF0E9EB602D0E82EFCD7AE
:105D3000C9CFB2F5B2EC2DF0A1EC2DF09E96C69E27
:105D400022C0C9FFFF0E9EB602D0E82EFCD79E9659
:105D5000C69E000EC96EFF0E9EB602D0E82EFCD77E
:105D6000C9CFB6F5B2EC2DF01200A1EC2DF09E9645
:105D7000C69E870EC96EFF0E9EB602D0E82EFCD7D7
:105D80009E96C69EAFC5C9FFFF0E9EB602D0E82EF6
:105D9000FCD79E96C69EB0C5C9FFFF0E9EB602D028
:105DA000E82EFCD79E96C69EB1C5C9FFFF0E9EB6D3
:105DB00002D0E82EFCD79E96C69EB2C5C9FFFF0E44
:105DC0009EB602D0E82EFCD7B2EC2DF0A1EC2DF05F
:105DD0009E96C69E23C0C9FFFF0E9EB602D0E82E37
:105DE000FCD79E96C69EB6C5C9FFFF0E9EB602D0D2
:105DF000E82EFCD7B2EC2DF01200A1EC2DF09E960F
:105E0000C69E870EC96EFF0E9EB602D0E82EFCD746
:105E10009E96C69E000EC96EFF0E9EB602D0E82E5C
:105E2000FCD79E96C69E800EC96EFF0E9EB602D00F
:105E3000E82EFCD79E96C69E800EC96EFF0E9EB6BB
:105E400002D0E82EFCD79E96C69E800EC96EFF0E2D
:105E50009EB602D0E82EFCD7B2EC2DF01200A1ECD9
:105E60002DF09E96C69E870EC96EFF0E9EB602D07E
:105E7000E82EFCD79E96C69E000EC96EFF0E9EB6FB
:105E800002D0E82EFCD79E96C69E000EC96EFF0E6D
:105E90009EB602D0E82EFCD79E96C69E800EC96E96
:105EA000FF0E9EB602D0E82EFCD79E96C69E800EB0
:105EB000C96EFF0E9EB602D0E82EFCD7B2EC2DF0D4
:105EC000120010A817D0A1EC2DF09E96C69E8F0E42
:105ED000C96EFF0E9EB602D0E82EFCD79E96C69ED7
:105EE000000EC96EFF0E9EB602D0E82EFCD7B2ECB3
:105EF0002DF0120063EC2EF0120010A82DD0A1ECB2
:105F00002DF09E96C69E23C0C9FFFF0E9EB602D0FE
:105F1000E82EFCD79E96C69E450EC96EFF0E9EB615
:105F200002D0E82EFCD7B2EC2DF0A1EC2DF09E961D
:105F3000C69E8F0EC96EFF0E9EB602D0E82EFCD70D
:105F40009E96C69E000EC96EFF0E9EB602D0E82E2B
:105F5000FCD7B2EC2DF01200A1EC2DF09E96C69E5F
:105F600023C0C9FFFF0E9EB602D0E82EFCD79E9636
:105F7000C69E010EC96EFF0E9EB602D0E82EFCD75B
:105F8000B2EC2DF0A1EC2DF09E96C69E910EC96E3E
:105F9000FF0E9EB602D0E82EFCD79E96C69EA50E9A
:105FA000C96EFF0E9EB602D0E82EFCD7B2EC2DF0E3
:105FB0001200A1EC2DF09E96C69E23C0C9FFFF0ED5
:105FC0009EB602D0E82EFCD79E96C69E810EC96E64
:105FD000FF0E9EB602D0E82EFCD7B2EC2DF01200D8
:105FE000A1EC2DF09E96C69E23C0C9FFFF0E9EB663
:105FF00002D0E82EFCD79E96C69E010EC96EFF0EFB
:106000009EB602D0E82EFCD7B2EC2DF01200A1EC27
:106010002DF09E96C69E910EC96EFF0E9EB602D0C2
:10602000E82EFCD79E96C69EA50EC96EFF0E9EB6A4
:1060300002D0E82EFCD7B2EC2DF01200A1EC2DF02E
:106040009E96C69E910EC96EFF0E9EB602D0E82E99
:10605000FCD79E96C69E000EC96EFF0E9EB602D05D
:10606000E82EFCD7B2EC2DF012000501256B266B53
:10607000276B286B899A400EC76E200EC66E9E96BF
:10608000C69E030EC96EFF0E9EB602D0E82EFCD748
:106090009E96C69E27C5C9FFFF0E9EB602D0E82E6B
:1060A000FCD79E96C69E26C5C9FFFF0E9EB602D09F
:1060B000E82EFCD79E96C69E25C5C9FFFF0E9EB64C
:1060C00002D0E82EFCD79E96C69EC952FF0E9EB601
:1060D00002D0E82EFCD7898A0F01C950FF0A01E1DE
:1060E000120005012E51130A05E005012E51170A71
:1060F0000CE012000501F00E256FFF0E266F0F0E4B
:10610000276F000E286F8EEF30F00501F00E256F1F
:10611000FF0E266FFF0E276F000E286F899A400E24
:10612000C76E200EC66E9E96C69E030EC96EFF0EEB
:106130009EB602D0E82EFCD79E96C69E27C5C9FF04
:10614000FF0E9EB602D0E82EFCD79E96C69E26C5B0
:10615000C9FFFF0E9EB602D0E82EFCD79E96C69EC3
:1061600025C5C9FFFF0E9EB602D0E82EFCD79E962D
:10617000C69EC952FF0E9EB602D0E82EFCD7898A71
:106180000F01C950FF0A1DE005012E51130A05E059
:1061900005012E51170A0BE012000501000E256FB4
:1061A000000E266F100E276F000E286F12000501DB
:1061B000000E256F000E266F000E276F010E286F50
:1061C00012000501256B266B276B286B05012E51EC
:1061D000130A05E005012E51170A0CE01200050113
:1061E000000E216F000E226F080E236F000E246F29
:1061F00003EF31F00501000E216F000E226F800EBB
:10620000236F000E246F21C500F122C501F123C5C3
:1062100002F124C503F125C504F126C505F127C502
:1062200006F128C507F189EC2AF000C125F501C166
:1062300026F502C127F503C128F5899A400EC76EDD
:10624000200EC66E9E96C69E030EC96EFF0E9EB6AB
:1062500002D0E82EFCD79E96C69E27C5C9FFFF0E2A
:106260009EB602D0E82EFCD79E96C69E26C5C9FFD4
:10627000FF0E9EB602D0E82EFCD79E96C69E25C580
:10628000C9FFFF0E9EB602D0E82EFCD79E96C69E92
:10629000C952FF0E9EB602D0E82EFCD7898AC9509B
:1062A000FF0A08E104C125F505C126F506C127F559
:1062B00007C128F5D8900501243323332233213335
:1062C0002151F00B216F21676DEF31F022676DEFE7
:1062D00031F023676DEF31F0246703EF31F00501F2
:1062E000100E2527E86A2623E86A2723E86A282370
:1062F0001200E86A05012E51130A06E005012E512D
:10630000170A0BE0020E120005012851000A03E1F2
:106310002751F00B07E0010E120005012851000A79
:1063200001E0010E120029C500F12AC501F12BC5BB
:1063300002F12CC503F125C504F126C505F127C5D9
:1063400006F128C507F138EC2CF003BF120079ECF8
:1063500031F0D8A40BEF32F0899A400EC76E200EB0
:10636000C66E9E96C69E060EC96EFF0E9EB602D0E3
:10637000E82EFCD7898A899A9E96C69E020EC96E1F
:10638000FF0E9EB602D0E82EFCD79E96C69E27C56D
:10639000C9FFFF0E9EB602D0E82EFCD79E96C69E81
:1063A00026C5C9FFFF0E9EB602D0E82EFCD79E96EA
:1063B000C69E25C5C9FFFF0E9EB602D0E82EFCD7AB
:1063C0009E96C69E000EC96EFF0E9EB602D0E82EA7
:1063D000FCD7898A899A9E96C69E050EC96EFF0EC5
:1063E0009EB602D0E82EFCD79E96C69EC952FF0EDE
:1063F0009EB602D0E82EFCD7C9B0F4EF31F0898AFE
:106400000501100E2527E86A2623E86A2723E86A93
:10641000282393EF31F01200899A400EC76E200EA8
:10642000C66E9E96C69E060EC96EFF0E9EB602D022
:10643000E82EFCD7898A899A9E96C69EC70EC96E99
:10644000FF0E9EB602D0E82EFCD7898A0501256B87
:10645000266B276B286B1200899A400EC76E200EA0
:10646000C66E9E96C69E050EC96EFF0E9EB602D0E3
:10647000E82EFCD79E96C69EC952FF0E9EB602D04D
:10648000E82EFCD7C9CF37F5898A1200899A400EC9
:10649000C76E200EC66E9E96C69EB90EC96EFF0EC2
:1064A0009EB602D0E82EFCD7898A1200899A400E47
:1064B000C76E200EC66E9E96C69EAB0EC96EFF0EB0
:1064C0009EB602D0E82EFCD7898AFF0EE82EFED7B2
:1064D000120079EC31F0D8A41200899A400EC76EF0
:1064E000200EC66E9E96C69E030EC96EFF0E9EB609
:1064F00002D0E82EFCD79E96C69E27C5C9FFFF0E88
:106500009EB602D0E82EFCD79E96C69E26C5C9FF31
:10651000FF0E9EB602D0E82EFCD79E96C69E25C5DD
:10652000C9FFFF0E9EB602D0E82EFCD79E96C69EEF
:10653000C952FF0E9EB602D0E82EFCD7898A0F0101
:10654000C950FF0AD8A466EF33F00501FE0E376F7D
:1065500030A03799BBEC2DF0AFC538F5B0C539F593
:10656000B1C53AF5B2C53BF5B3C53CF5B4C53DF58B
:10657000B5C53EF50784B6C166F1B7C167F1B8C1CC
:1065800068F1B9C169F14BC14FF14CC150F14DC136
:1065900051F14EC152F157C159F158C15AF11CEC99
:1065A00021F000C13FF501C140F502C141F503C131
:1065B00042F505016167E4EF32F06267E4EF32F023
:1065C0006367E4EF32F06467E8EF32F0F5EF32F042
:1065D00061C504F162C505F163C506F164C507F143
:1065E00038EC2CF003BF66EF33F059C143F55AC1C4
:1065F00044F5B9C545F5BAC546F507940501110E30
:10660000326F899A400EC76E200EC66E9E96C69E49
:10661000060EC96EFF0E9EB602D0E82EFCD7898A00
:10662000899A9E96C69E020EC96EFF0E9EB602D035
:10663000E82EFCD79E96C69E27C5C9FFFF0E9EB6C4
:1066400002D0E82EFCD79E96C69E26C5C9FFFF0E37
:106650009EB602D0E82EFCD79E96C69E25C5C9FFE1
:10666000FF0E9EB602D0E82EFCD725EE37F0322F73
:1066700002D046EF33F09E96C69EDECFC9FFFF0ED6
:106680009EB602D0E82EFCD737EF33F0898A899A7C
:106690009E96C69E050EC96EFF0E9EB602D0E82ECF
:1066A000FCD79E96C69EC952FF0E9EB602D0E82E1B
:1066B000FCD7C9B051EF33F0898A0501100E2527A8
:1066C000E86A2623E86A2723E86A2823120021C5FE
:1066D00000F122C501F123C502F124C503F1899A15
:1066E000400EC76E200EC66E9E96C69E0B0EC96EDD
:1066F000FF0E9EB602D0E82EFCD79E96C69E02C123
:10670000C9FFFF0E9EB602D0E82EFCD79E96C69E0D
:1067100001C1C9FFFF0E9EB602D0E82EFCD79E969F
:10672000C69E00C1C9FFFF0E9EB602D0E82EFCD760
:106730009E96C69EC952FF0E9EB602D0E82EFCD78A
:1067400025EE37F00501100E326F9E96C69EC95297
:10675000FF0E9EB602D0E82EFCD7C9CFDEFF322F47
:10676000A5EF33F0898A1200899A400EC76E200E79
:10677000C66E9E96C69E900EC96EFF0E9EB602D045
:10678000E82EFCD79E96C69E000EC96EFF0E9EB6E2
:1067900002D0E82EFCD79E96C69E000EC96EFF0E54
:1067A0009EB602D0E82EFCD79E96C69E000EC96EFD
:1067B000FF0E9EB602D0E82EFCD79E96C69EC9520A
:1067C000FF0E9EB602D0E82EFCD7C9CF2DF59E96BF
:1067D000C69EC952FF0E9EB602D0E82EFCD7C9CF86
:1067E0002EF5898A120004EC2BF0B9C5E8FFD70812
:1067F00002E304EC2BF0B9C5E8FFC80802E304EC9F
:106800002BF0B9C5E8FFB90802E304EC2BF0B9C5D9
:10681000E8FFAA0802E304EC2BF0B9C5E8FF9B08E7
:1068200002E304EC2BF046EC32F0F29CF29E8B94E7
:10683000C69AC2909482948C720ED36ED3A4FED763
:1068400089968A909390F29AF2949D909E909D9250
:106850009E92F298F29261EC2FF0FF0EE8CF00F0DA
:10686000E82EFED7002EFCD7F290F286815081A848
:106870003CEF34F0F29E0300F296F290010E306E7F
:0A688000038025EC2BF056EF0BF01F
:10BF0000E844F926000C160C2B0C3F0C520C640C68
:10BF1000760C860C960CA50CB30CC10CCF0CDC0C6B
:06BF2000E80CF40C000C1B
:0200000400F00A
:0100C800FE39
:00000001FF
